:020000040800F2
:10500000D81B0020D55000088D8C0008658300084F
:105010000000000000000000000000000000000090
:10502000000000000000000000000000E1990008FE
:10503000000000000000000089920008F99A0008B2
:10504000E7500008E7500008E7500008E750000864
:10505000E7500008895D0008E7500008E7500008A5
:1050600000000000E7500008B15C0008E7500008AD
:10507000E75000087D88000800000000E7500008A5
:1050800000000000E75000080000000000000000E1
:10509000E750000800000000E7500008E750000853
:1050A000E7500008E7500008E7500008A5A50008F1
:1050B000E7500008E7500008000000000000000072
:1050C0000348854600F040FD0048004725B9000828
:1050D000D81B00200448804704480047FEE7FEE74D
:1050E000FEE7FEE7FEE7FEE7959B0008C1500008DB
:1050F00030B50B46014600202022012409E00D4670
:10510000D5409D4205D31D469540491B25469540F7
:1051100040191546521E002DF1DC30BDF0B51FB40C
:105120000646002082B005464024019100901BE015
:10513000019922460F46304600F0F0FB049A059B89
:10514000801A994110D310461946224600F0D6FB2A
:10515000361A8F410197224601200021009F00F05E
:10516000CDFB38184D4100902046641E0028DFDC3E
:10517000019B00982946324607B0F0BD03460B4319
:105180009B0703D009E008C9121F08C0042AFAD2FD
:1051900003E00B780370401C491C521EF9D2704783
:1051A000D2B201E00270401C491EFBD270470022BF
:1051B000F6E710B513460A4604461946FFF7F0FF16
:1051C000204610BD30B504460020034600E05B1CBD
:1051D000934203D2E05CCD5C401BF8D030BDF8B503
:1051E00002464A40D40F42004B0052085B089A42E4
:1051F00002D20246084611464A0023D0C30D4A0097
:10520000DDB2120EAD1A202D35DA49020126490A07
:10521000F6058A19002C00D0524220214F1B11465E
:10522000B9402A411018C20D9A4221D0002C17D043
:10523000012D08DCDA05801AD20F8019D207DBB203
:1052400000F098FBF8BDDA05801A012340001B0628
:10525000C01880185A428018CA0F1043490007E04E
:105260004908C2071143DA05801A801940088018DE
:1052700000F078FBF8BD61000122511A001BF7E72E
:105280000122D2075140AAE70122D2075040A6E7E7
:10529000024670B54A40D30FDB0740002DD04A00CC
:1052A0002AD0010E140E000212020919400A520AF5
:1052B0008418E50104465443000A120A2E045043A0
:1052C000A4194219200CC543AA18120C0125AD03DC
:1052D000521C521912047F39240400D0521C10436E
:1052E00001D44000491EC2B20C06C0092018401C5F
:1052F0004008802A02D003E0002070BD4008400032
:10530000002900DA0020184370BD70B502464A40FB
:10531000D50F40004A00ED0740085208002814D07D
:10532000002A12D0C40DD30D41020120C005520243
:10533000490A520AE41A091812187D34914201D31D
:10534000641C00E04900002C01DA002070BD00233D
:10535000914201D3891A0343400849000028F7D13C
:1053600000290AD0914202D10121C90705E09142EA
:1053700001D2012101E00121C943E005C018401913
:1053800000F0F0FA70BD420005D04200120E524209
:105390008A4201DB00207047C905081870470000E9
:1053A000F0B507460846584087B0C00F0490480043
:1053B0000E46590040084908BC1A884105D23846B3
:1053C00031461E4617460B46024658004008104319
:1053D0004CD0300D039040055900400D490D05900B
:1053E000401A0290402872DA18030121000B0905C7
:1053F0000843019004980092002805D00199524278
:105400000020884100920190029840210A1A0199D7
:10541000009800F073FA05460C466B4607CB00F087
:105420008EFAC0197141039A0E0D0023D71756400A
:105430001A467A40164344D0049A002A2DD0029A84
:10544000012A039A15DC1205C01A9141012636057E
:10545000001C7141D20F059ED20700930192029663
:105460002A46234600F0CCFA07B0F0BD3846314654
:10547000FAE71605224A0F46B218C01AB7410121B1
:105480000905001C4F4100187F4111461818794149
:10549000E20F10436D19644113E0E2076D081543F4
:1054A0006408C2071443039A01261205C01A9141E9
:1054B0003605001C7141CE07400830434908C0182A
:1054C00051412A46234600F08EFACDE7FFE70498C3
:1054D00001224000C117121A00238B410498314663
:1054E000C417381AA141EEE730B40124E407634041
:1054F00030BC55E730B40124E407614030BC4FE7CD
:105500000000E0FFF0B51FB488B00B9909980024A3
:1055100048400999C00F490049080991C0070B99F3
:105520000090490049080B9109990898A64608433C
:105530001CD00B990A98084318D009980124400000
:10554000420D4800410D099824050003000B20433B
:1055500009900B980003000B20430B9050181C4936
:105560004018002201901446104605E00020014634
:105570000DB0F0BD032801DA034600E003239C468A
:10558000C11A0AAE0AE05F0008ADED5B4F00F75BA1
:105590007D430027AA187C41491C5B1E6145F2DD52
:1055A000410004AB5A522104120C0A43240C401C43
:1055B0000828DFDB01980290009970460191009065
:1055C000059B049A0799069800F01AFAD0E70000A4
:1055D0000DFCFFFFF0B50C465C4085B0E40FE4071E
:1055E00003944C000026640859009446490802467A
:1055F0000296224321D062460A431ED06200570D14
:105600004A000E032303550D012402462C492405AC
:10561000781B1B0B360B4018234326436146009032
:105620001C46501AB44103D30098401C009002E07D
:10563000921800985B41002803DA0020014605B06B
:10564000F0BD0020012109050746864611E06446A9
:105650001D46141BB54106D36546521BB341744623
:1056600007430C43A646CD07400849082843921833
:105670005B4105460D43EAD11046184313D06046FE
:10568000194650407140084306D06046101AB34195
:1056900006D20122002306E000220123DB0702E0FC
:1056A0000122D2435310009874460105381C614111
:1056B000029C039D0019694100F095F9BFE70000C5
:1056C000FD03000070B54B005B0803430BD04B009B
:1056D0005C0D002633466542B341D417AD1AA34191
:1056E00002DB0020014670BD12053018514170BD2B
:1056F000C217C10F504010B54018CA0796230021A9
:1057000000F038F910BD10B500229623114600F0C4
:1057100031F910BD0EB5C217C10F5040CA0740186D
:105720000021054B0293019200910A460B4600F0BE
:1057300067F903B000BD0000330400000EB5054951
:105740000291002100910A460B46019100F058F9A0
:1057500003B000BD33040000C20F4100400201232A
:10576000400ADB05D207090EC0187F2901DA0020A4
:105770007047962903DC9623591AC84001E09639F0
:105780008840002AF4D04042704741004002012284
:10579000400AD205090E80187F2901DA00207047DF
:1057A000962903DC9622511AC840704796398840E2
:1057B0007047000070B5CD0F4A0009030123090BA3
:1057C0001B0519430B4BED070024520D9A4201DAD9
:1057D000002070BD074B34339A4203DC9A1A00F064
:1057E0009DF802E00449511888402C43F1D0404212
:1057F00070BD0000FF030000CDFBFFFF4A0009035E
:105800000123090B1B051943094B10B5520D9A4290
:1058100001DA002010BD064B34339A4203DC9A1A99
:1058200000F07CF810BD03495118884010BD0000FD
:10583000FF030000CDFBFFFFC20FD207400040086E
:105840000BD0C10D0723DB01C91840020905400A2E
:105850001143C208400711437047002001467047BA
:1058600010B5002904DB0124E40740428C412146A5
:10587000002B04DB1C460123DB075242A3418B4271
:1058800000D1824210BD000010B5002904DB0124C4
:10589000E40740428C412146002B04DB1C460123D7
:1058A000DB075242A341994200D1904210BD000053
:1058B000CB0FDB07490010B5490802460A4307D061
:1058C0000A0D07240903E401090B121B002A01DC5D
:1058D000002010BDC900440F0C43C100E018D205E0
:1058E000801800F03FF810BD0122D207002800DB2D
:1058F000101A002900DB511A8142704710B5202A86
:1059000004DB0146203A9140002010BD9140202345
:105910009C1A0346E3401943904010BD10B5202A5D
:1059200004DB0846203AD040002110BD0B46D3408E
:10593000D0402024A21A91400843194610BD10B54A
:10594000202A06DBCB170846203A1041C1170B432B
:1059500006E00B461341D0402024A21A9140084390
:10596000194610BD002904DA401C490001D1400845
:105970004000704770B40024050C05D110240004C9
:1059800002D1002921D01124050E01D100020834D2
:10599000050F01D10001241D850F01D18000A41C39
:1059A000002801DB4000641C002908D020252E1BA4
:1059B0000D46F540A14000D00121294308430106CE
:1059C0001B1B000ADB1D02D5002070BC7047DB05E5
:1059D000181880180029F8DA401C4900F5D170BC6D
:1059E00040084000704710B5002B08DA0024401C26
:1059F000614192185B411A4301D14008400010BD3B
:105A0000F0B51FB482B005460C0003D0084604F080
:105A100083FE02E004F080FE203002460090214622
:105A20002846FFF76BFF049B059A04460F46184370
:105A30001143084314D0184610431BD0009840214E
:105A40000A1A18460599FFF769FF05460E46009A9F
:105A500005990498FFF752FF084305D0012004E0A0
:105A60002046394607B0F0BD0020C11705430E435C
:105A70002C43374300990E986305401A7905E40AD0
:105A800000220C43FD0A0A3002D500200146E9E756
:105A90000105101969410C9C0D9D00196941FFF722
:105AA000A2FFDFE7FEB500231A461B1A8A4103DB7B
:105AB0000020014603B0F0BD4A000D0301212D0B6B
:105AC0000905520D0D43D10702D100186D41521E38
:105AD0005110FF31FF310131002704463E46384660
:105AE000009701910246012100200905FFF716FFEA
:105AF000C3197141F818324684468E464A416146C0
:105B00002846611A904104D36046241A954176468E
:105B10001F46241900986D41401C00903428E1DD97
:105B2000F91930467041091BA84103D20022D24323
:105B3000134601E00022134601980105381C71410B
:105B4000FFF751FFB6E70000064C0125064E05E0C1
:105B5000E36807CC2B430C3C98471034B442F7D38E
:105B6000FFF7B2FA18C8000838C8000870B58C18DA
:105B70000578401C6B075B0F01D10378401C2A118C
:105B800006D10278401C03E006780E70401C491CC8
:105B90005B1EF9D12B0705D40023521E0DD40B70C8
:105BA000491CFAE70378401CCB1A921C03E01D78CD
:105BB0000D70491C5B1C521EF9D5A142D8D30020A0
:105BC00070BD000038B50446064805490068FFF777
:105BD0008FFA604300E0401E00900028FBD138BDE2
:105BE00040420F0078010020F8B504460068816843
:105BF0008907890F012902D10168C90722D181686B
:105C0000114A10261140012500290ED1816829432F
:105C100081600120FFF7D6FF01F008F807460CE08D
:105C200001F004F8C01B0A2807D9606D3043606595
:105C3000A06D2843A0650120F8BD20680068C0431E
:105C4000C007EDD10020F8BD170000801FB50B483C
:105C500000900B4801900B4802900B480390694656
:105C60000A4805F04FF90A4A08481146083905F074
:105C700037F800F04FFA002004B010BD21C600082C
:105C8000FDC500085DC600085BC600088401002051
:105C90001000002010B500231A4603E0845CE318CE
:105CA0009BB2521C8A42F9D3D84380B210BD000087
:105CB00010B5034800F076FD024800F073FD10BDFA
:105CC000781700203017002030B5446C1C252C407C
:105CD0000125A540046C6560046863608368102B2F
:105CE000036803D099600068C26030BD9A600068A4
:105CF000C16030BD1449012048720A4602205E325C
:105D0000507203203C3A507204200E3A50720F48F1
:105D10000D4B0078087022310870203108770C494B
:105D20005A1C087858714978997123331871597140
:105D3000203318775977107551751A461E32107531
:105D40005175107651767047DC1100202701002034
:105D50004801002010B503F019FE202003F0C2FE18
:105D6000012005F039FB002003F0BCFE044805F0DB
:105D7000D7F9044805F086FC002005F0BBFC10BDF7
:105D8000E800002083800000F8B50520012100070D
:105D900000F038FF0025174C002800D06560164E33
:105DA0000221304600F02EFF00281BD10120207078
:105DB0001248808F00280ED00127BF0200223946EA
:105DC000304600F02CFF0A2004F0FAFE012239468A
:105DD000304600F024FF0A48656000880A214843E5
:105DE00008490880012000F045FE022000F042FE34
:105DF000F8BD00006401002000040050DC0D00200C
:105E000034010020460100207047000010B5084909
:105E100000224A6107494B684C1523434B604B688D
:105E2000082423434B60C009C001026010BD00007C
:105E3000C0170020002002407FB500250C46064612
:105E4000039500F0E7FDE009029003A90196009593
:105E5000684600F077FD002804D000F0AFFD002078
:105E600004B070BD00F0AAFD0120F9E710B50023D1
:105E700002E0C45CCC545B1C9342FAD310BD00001A
:105E800010B5214A00219069C305204804D5416915
:105E9000022319434161911593699B0505D5436917
:105EA0000124234343616302194393695B0505D5CC
:105EB0004369082423434361E301194393691B05A4
:105EC00005D543690424234343616302194393695D
:105ED0009B0405D54369102423434361630219439E
:105EE00093699B0304D5446920231C4344611943EF
:105EF0009369DB0305D54369402423434361A00232
:105F00000143916110BD000000200240C017002035
:105F100070B5054600F08AFE0646184C0AE0681C7B
:105F200008D0002D04D000F081FE801BA84201D9CA
:105F3000032070BDA069C007F1D1A069800701D519
:105F40000220A061A069C00511D4A06980050ED40B
:105F5000A06940050BD4A069000508D4A06980049D
:105F600005D4A069800302D4A069C00303D5FFF75C
:105F700087FF012070BD002070BD0000002002409E
:105F8000F8B51746002605460C4600F043FD09E02B
:105F900029460220226800F01FFD002804D1241D9C
:105FA0002D1D361DBE42F3D300F008FDBE4201D2C6
:105FB0000020F8BD0120F8BD10B5084902460020B8
:105FC000054B497905E044001C5B944203D0401C1A
:105FD000C0B28842F7D310BD8213002070000020A9
:105FE00010B500F014FE10BD10B5094801F03EF8E0
:105FF00080B2FFF7A3FB074A074BFFF783FA0022A3
:10600000064BFFF7E7FAFFF7F9FB80B210BD00007F
:10601000E4150020F853E3A59B843E4000408F40E8
:1060200070B5374C3548A0842146364820310A796E
:1060300002754979417534490A7802764978417682
:1060400030490520133148720A2005F00BFB7D20F2
:10605000C00005F021FB2B49002213310C2005F074
:10606000EBFB00210C2005F0F9FB022005F04AFBB8
:10607000264D00210F2005F075FA2842A063F8D0C4
:10608000A06B411C37D0400434D58122D2010021BD
:106090000F2005F0A6FB0021102005F063FA410651
:1060A0001848490E0022C73005F092FA154DC73541
:1060B000687A05281ED102221349681DFFF782F86D
:1060C000002817D10E48AE7C66710422691C50303E
:1060D000FFF754F829461331084672000D466B301D
:1060E000FFF74CF86079294642000948FFF746F867
:1060F0000320207070BD04F083FB00002497000093
:10610000700000203D1200204801002000D027240C
:106110009A13002010B5144C144822461032114630
:10612000083904F0DDFD0022114BE168A068FFF79B
:1061300051FA104A104B05F003FD00220F4BFFF7F8
:10614000D9F900220E4BFFF7DDF9FFF7B1FB206014
:1061500000221346E168A068FFF782FB01D02068A7
:1061600010BD0020206010BD000000208401002030
:1061700000AA8F406C45D9CC955BC83F0000F03F2A
:1061800040A5E54010B5084800F096FA0A210648F7
:1061900000F032FA044800F01DF9800503D50248EA
:1061A00000F01AF980B210BD88150020F8B52F4D07
:1061B00000220121284600F032FDFFF7E3FFFFF740
:1061C000A2FA2B4E3146FFF7A0F82A4C0122A0601C
:1061D0001146284600F023FD2749A0680025884283
:1061E0003EDB2078254F002815D02570FFF7CAFF29
:1061F000FFF789FA3146FFF788F8A060FFF71CFB2C
:1062000000223B46FFF770F900221D4BFFF77AF999
:10621000FFF74EFB6060A068FFF70EFB00223B46D5
:10622000FFF762F9174A184BFFF76CF906460F465D
:106230006068FFF701FB134A144B5242FFF762F903
:1062400032463B46FFF7ACF8FFF732FB104960607F
:10625000884201DD616004E0FF21C905C84200D326
:1062600065606068FFF791FAC0B2F8BD00040050A5
:1062700000401B44480000200000604000000C402B
:1062800000E064403333333333B33040CCCCEC3FA5
:106290000000C842F8B5054604464035287C002673
:1062A000012808D001202874206881688907890F97
:1062B00001290ED101E00220F8BD0168C90708D00C
:1062C000606D202108436065012600202874304657
:1062D000F8BD616DFF2201329143022211436165D5
:1062E000C1688907890F0091C16889088900C16068
:1062F0002068816892071143816000F097FC07468F
:106300000EE000F093FCC01B0A2809D9606D022141
:106310008843102108436065002028740120F8BDDF
:10632000206880680028ECDB2068C168009A11436F
:10633000C160606D80088000401C6065C5E700009A
:10634000F8B506460D464036317C01290DD00121B5
:10635000317401688A68520709D5416D20221143C2
:106360004165002030740120F8BD0220F8BD174BB4
:106370006A68D80547109A42154C8A6A2B6812D071
:106380005B035B0B1A438A622968490305D5A16840
:106390000143A1600A20FFF715FC2868800312D58D
:1063A000A06838430EE05B035B0B9A438A6229685E
:1063B000490302D5A1688143A1602868800302D502
:1063C000A068B843A06000203074F8BD0110000040
:1063D00000270140406D70470068006C7047000066
:1063E00070B5040006D0606D2646002540360028B2
:1063F00002D006E0012070BDA5653574204600F08E
:10640000D3F8606DC00603D421688868400705D5BD
:10641000606D1021084360653574EBE7606DFF2205
:106420000132904302221043606588688207920F10
:106430005B48012A02D10A68D2072BD10323626884
:106440009B079A4205D05B429A4202D05B009A4277
:1064500009D10A69920092080A6121680A69636891
:106460001A430A610CE00A69920092080A61816885
:106470000F229204914381608168626811438160B8
:106480002168CA6818239A43CA602168CA68A36849
:106490001A43CA6081680122520691438160816873
:1064A000A28E52061143816020688168C90004D41D
:1064B000816801221207114381602068C168394A4E
:1064C0001140C1602069E168022825D00020014305
:1064D000204620300278037B52035B001A431143AD
:1064E000226B1143A26992031143E269D203114363
:1064F0002268D3681943D160616A0A46FF3AC23AFA
:1065000005D0A26A11432268D3681943D16042784A
:106510000121012A02D00BE00420D8E700780028EE
:1065200023D0606D202210436065A06D0843A065F4
:10653000E06B012820681FD00169C90703D00169F9
:1065400049084900016120684169C908C9004161E1
:1065500020684169A26B11434161A565606D8008A7
:106560008000401C6065002070BD2068C268012367
:106570001B041A43C260DBE70269FF239B009A43B6
:10658000026120680269236CA66C1A43636C334372
:106590001A430261206802690A430261D3E70000DE
:1065A000002701401902FEFF10B586B004461421F1
:1065B0006846FEF7FCFD0E492068884216D10D485A
:1065C000416B421511434163C16A01221143C1620B
:1065D000C06A694610400590022000900320019097
:1065E000002002900520000700F050FA06B010BD10
:1065F0000024014000100240F8B5044640692546D9
:1066000040350E4608280BD02068C068C00709D066
:10661000606D202108436065002028740120F8BDCA
:10662000082700E00C2700F001FB009011E0701C2F
:106630000FD0002E05D000F0F9FA0099401AB042B0
:1066400007D9606D04210843606500202874032089
:10665000F8BD206800683842E9D0606D0121490228
:10666000084360652068C16809058A0F0C21002A6B
:106670001BD12022125D002A17D10268120714D5FF
:10668000826853070122002B08DB43688B43436079
:10669000606D130298431043606506E0606D20232F
:1066A00018436065A06D1043A065A069002801D162
:1066B000206801600020F8BD70B504462168002004
:1066C0008968490721D425464035297C01291CD0F9
:1066D00001212974E169012904D02046FFF784FAD9
:1066E000002811D1616D0A4A1140FF220132114385
:1066F00061650021A165297422681C21116021684F
:106700008A6804231A438A6070BD022070BD0000AD
:10671000FEF1FFFF30B5014620314A790023022AFD
:1067200004D00422C2630B71012030BD02681468DA
:106730000E25AC4314600268146864086400146099
:10674000446C1C22144001221546006CA540456093
:106750004A7118460B7130BD70B5002401462031D6
:106760004A79022A03D00421C163012418E0026897
:1067700013680E25AB431360026813685B085B0067
:106780001360436C1C221340012215469D40036C8C
:106790005D604A7100220A71816B002900D0884730
:1067A000204670BDF0B4016C0D6801680C68466C41
:1067B0001C2304221E401746B7402F420ED0670705
:1067C0000CD50C68A40602D40C6894430C60416C90
:1067D00019408A40016C4A60016B1AE00227B740F9
:1067E00002462F402032002F17D0A70715D50C687E
:1067F000A40605D40C680A25AC430C600121517134
:10680000446C02211C40036CA140596000211171AD
:10681000C16A002918D0F0BC08470827B7402F42AA
:1068200012D0240710D50C680E25AC430C60446CC4
:1068300001211C400B46A340046C6360C16351718D
:1068400000211171416BE4E7F0BC704770B50400A2
:106850003CD01F48256814212818FEF749FC800009
:1068600060641C48206402212046203002464171A9
:1068700029681948E3680140A068666918432369DC
:1068800033431843A3691843E3691843236A184341
:10689000084328600121A0688903884210D00D4870
:1068A0008030836A656C1C210D400F26AE40B343D7
:1068B0008362656C63680D40816AAB400B43836201
:1068C0000020E06301215171107170BD012070BD85
:1068D000F8FFFDBF000002400F80FFFFF8B504463F
:1068E0008C46203001790025012909D00126067146
:1068F00041790027012905D0077102252846F8BDF6
:106900000220F8BD02214171E7632068016849084F
:106910004900016061462046FFF7D6F9206B002848
:106920002068016801D00E2205E004229143016035
:10693000206801680A221143016020680168314320
:106940000160DBE7F8B51A4E0546307C0F4601289A
:1069500007D0012030741748FFF7DAFA010002D09F
:1069600021E00220F8BD0020C04338606C6814E0CC
:106970002046FFF74BFA0F48FFF7CAFA01460E48C8
:10698000426808239A434260426843159A43426032
:10699000002901D03C6006E08034A8686A68C00124
:1069A0008018A042E4D8002030740846F8BD0000EA
:1069B000C017002050C30000002002400548416875
:1069C00002221143416041680122114341600020CD
:1069D0007047000000200240F8B50C4C1646207CA1
:1069E0000F46012808D0012020740948FFF790FACB
:1069F0000025002802D006E00220F8BD65613E6057
:106A00000348FFF785FA2574F8BD0000C017002081
:106A100050C3000011484168C9070BD0EFF3108143
:106A200072B60F4AC2600F4AC26081F31088416893
:106A3000C9070ED1416889070DD5EFF3108172B6F1
:106A4000094A0261094A026181F31088406880079F
:106A500001D501207047002070470000002002404F
:106A6000EFCDAB8905040302BFAE9D8C1615141340
:106A70007047000010B504494A69024202D04861DB
:106A8000FFF7F6FF10BD000000040140FCB5002335
:106A90000124A2E027462A469F403A406FD04D6825
:106AA000012D05D0022D03D0112D01D0122D16D1AC
:106AB00085680326AC465D00AE46AE406546B543EC
:106AC000AC46CE687546AE4065462E438660466845
:106AD0000D79BE43ED06ED0F9D4035434560C66818
:106AE0005F000325BD40AE46AE4335468E68BE40CE
:106AF0002E43C6604E68022E01D0122E14D1DE083D
:106B0000B60036180196366A5D07B446EE0E0F25BC
:106B1000B54000966646AE43B4460D69009EB5404A
:106B200066462E43019D2E6206687546AE430D797A
:106B3000AD07AD0FBD40354305604D68ED004BD549
:106B4000294D6E6B26436E639E08284DB60075195D
:106B5000AC46AD689E07360F0F27B740BD430527EB
:106B60003F07B84201D1002715E0214FB84201D1BB
:106B7000012710E01F4FB84202D102270BE02BE0A3
:106B80001D4FB84201D1032705E01C4FB84201D187
:106B9000052700E00627B7402F436546AF60184D34
:106BA0002E684F689643FF0300D516432E606E682B
:106BB0004F689643BF0300D516436E60AE684F68BA
:106BC0009643FF0200D51643AE60EE684F689643C9
:106BD000BF0200D51643EE605B1C0A681546DA401A
:106BE00000D057E7FCBD000000100240000001404B
:106BF0000004005000080050000C0050001C005021
:106C0000000401400069084000D00120704742693B
:106C100013460B401B0491430B4383617047002ACA
:106C200001D081617047816270470000014880682F
:106C3000704700006C0100200248816802788918C2
:106C4000816070476C01002010B50848002401687D
:106C5000402211430160204600F00AF8002801D0CC
:106C6000012401E000F04CFA204610BD0020024053
:106C700070B504460D4D7D202978C000FEF738FA26
:106C800001460B480068FEF733FA00F035FF002894
:106C900009D1042C07D200222146401E00F058FAE8
:106CA00000206C6070BD012070BD00006C010020F0
:106CB0007801002070477047F8B5654CA078401CFB
:106CC000A07001202071A08B401CA0836148008827
:106CD00002F0C4FE208AFEF716FD01467F20C005A3
:106CE000FEF713FB5C4D06462968FEF778FA28602C
:106CF0000120A16AC005814201DA084603E030465E
:106D0000FEF7C2FAA062FF21C9050025C84200D3E0
:106D1000A562607800280BD102215048FFF772FF6E
:106D200002004F494F4817D00022FFF778FFA563B4
:106D300002214A48FFF766FF4B4E002855D0A56355
:106D4000B08AFEF7E0FC444F3968FEF7CDFD5FD214
:106D50004649012008705DE00122D1034148FFF758
:106D60005EFF208AFEF7CFFC01467F20C005FEF7BC
:106D7000CCFAA16BFEF733FA3D49A0638842D7DD18
:106D800039480127F926403000900A213046FEF7A5
:106D9000AFF9002903D132493248FFF721F9022126
:106DA0002E48FFF72FFF002801D0002701E0002F19
:106DB00012D102212948FFF725FF00280CD104F049
:106DC00087FE00990120888005F0DEFB642003F037
:106DD000F7FE29492748C8600A2003F0F1FE304633
:106DE000761EF6B20028D0D1A2E7208AFEF78BFCEF
:106DF00001467F20C005FEF788FAA16BFEF7EFF988
:106E00001E49A06388429BDB1B491A48C86097E76C
:106E100016480570708F401EFEF76AFC3968FEF751
:106E200063FD06D86079002803D015490120087059
:106E300001E013480570708FFEF765FC3968FEF7B6
:106E400053FD04D26079002801D004F005FEF8BD9E
:106E5000240100209200002068010020000400505E
:106E60000080000000000050DC0D002076000020B3
:106E7000000040400400FA0500ED00E00000A040E2
:106E800083000020704770B5040010D00220254612
:106E90002035A873204601F0F9FCA87B032805D013
:106EA000204600F0B9F80020A873687370BD012077
:106EB00070BD7047704710B5044600680168C9434B
:106EC000C90708D18168C943C90704D101214160BC
:106ED0002046FFF7F1FE20680168C943890708D4FE
:106EE0008168C943890704D4022141602046FFF725
:106EF000E1FE20680168C943490708D48168C94395
:106F0000490704D404214160204600F0F7F82068C6
:106F10000168C943090708D48168C943090704D433
:106F2000082141602046FFF7ADFF20680168C94392
:106F3000C90608D48168C943C90604D41021416038
:106F40002046FFF7B8FE20680168C943890608D4C7
:106F50008168C943890604D4202141602046FFF797
:106F6000A9FF20680168C943490608D48168C9435C
:106F7000490604D4402141602046FFF79AFF10BD26
:106F8000F8B5040005D025462035A87B002802D09E
:106F900006E00120F8BD00206873204600F04EF89E
:106FA0000220A8732068C26884466368012B01D15F
:106FB0000620824316486169814202D007204003BF
:106FC0008243002B01D1D82082431248A668024098
:106FD00018463043676A266A3E433043A66A304308
:106FE0001043002B02D0012B04D005E02369E26995
:106FF0001A4300E0E2681043054A914202D0A269B8
:10700000114308436146C8600120A8730020F8BD01
:10701000FFFF0000F8F119FF10B50068054988422C
:1070200007D10548816B4900490881630D2000F0B4
:1070300073F810BD007C00400010024010B50068DD
:10704000084988420CD10848816BC204114381630E
:10705000002201210D2000F07BF80D2000F06CF8DB
:1070600010BD0000007C0040001002400068C069B4
:1070700070470000F8B50446022025462035174623
:10708000A8731D480268C3041A4302602068C268DE
:107090009B121A43C26020680269012632430261D2
:1070A000226810205060206881611021204601F084
:1070B0005DFC03281FD021680820486020684761D4
:1070C0000821204601F052FC032814D0204601F08C
:1070D000DDFBA87B03280ED02068816831438160E6
:1070E000206801693143016120680169042211436C
:1070F0000161AE730020F8BD00040140704700003C
:107100000448416B012211434163816B0204114326
:107110008163704700100240002809DBC106C90ED8
:107120000120884003490860BFF34F8FBFF36F8F82
:107130007047000080E100E0002805DBC106C90EB1
:1071400001208840014908607047000000E100E02C
:1071500010B503F033FB10BD02494A6882434A6010
:10716000704700000070004002480168821511431A
:10717000016070470070004002494A6802434A605B
:10718000704700000070004005480168022211436A
:1071900001600448016904221143016130BF704756
:1071A0000070004000ED00E0F0B5154A1368154D81
:1071B00054152D6A2340ED07ED0F002B04D0002D50
:1071C00002D01668A64316601668B608B6000643D5
:1071D00016600D48076904263743076101290DD061
:1071E00040BF20BF20BF0169B1430161002B04D023
:1071F000002D02D0106820431060F0BD30BFF2E7D0
:10720000007000400000014000ED00E0F8B50446C9
:1072100000780027534D800671D5524E403EB06B2A
:10722000C00004D4B06BA9050843B06301274E48E1
:107230000168C90511D40168821511430160FFF787
:10724000F5FC009005E0FFF7F1FC0099401A642876
:1072500037D845480068C005F5D5326803210905CF
:1072600060680A400140914208D08103890F0329D8
:1072700004D13168890301D50120F8BD2A690321B1
:1072800009040A4022D0084090421FD0207880068E
:107290001CD528692A6988430121C9040A432A6147
:1072A0002A698A432A612861C0050FD5FFF7BEFC11
:1072B000009008E0FFF7BAFC0099411A2B48814280
:1072C00001D90320F8BD28698005F3D561688803DA
:1072D000800F032805D132680005824301400A432C
:1072E0003260286903226168120411400843286152
:1072F000002F04D0B16B012000078143B1632078D7
:10730000C00705D0E868A168800880000843E860ED
:107310002078800705D5E8680C218843E168084398
:10732000E8602078400706D5E86803218902884391
:1073300021690843E8602078000706D5E868032142
:107340000903884361690843E8602078000606D590
:10735000E868032189048843A1690843E8600020A4
:10736000F8BD00004010024000700040881300008B
:10737000F8B50E46050038D05E480068C007C00F5B
:10738000B04214D25B4C206840084000304320607B
:10739000FFF74CFC074605E0FFF748FCC11B5648C9
:1073A00081427AD82068C007C00FB042F4D1287853
:1073B000524C800705D5E068F0218843A96808434E
:1073C000E0602878C00752D06868022806D00328F9
:1073D00007D0216801280AD0890504E021688903C3
:1073E00001E021688901002903DB0120F8BD49077C
:1073F000F9E7E168890889000143E160FFF716FCBD
:107400000746686802280AD0032814D001281ED035
:1074100029E0FFF70BFCC11B374881423DD8E068EB
:107420000007800F0228F4D121E0FFF7FFFBC11B0A
:107430003148814231D8E0680007800F0328F4D139
:1074400015E0FFF7F3FBC11B2B48814225D8E0680C
:107450000007800F0128F4D109E0FFF7E7FBC11B0B
:107460002548814219D8E0680007800FF5D12148EE
:107470000168C907C90FB14217D901684908490015
:1074800031430160FFF7D2FB074608E005E0FFF754
:10749000CDFBC11B1848814201D90320F8BD154816
:1074A0000068C007C00FB042F1D12878400706D568
:1074B000E068072109028843E9680843E06028780A
:1074C000000707D5E0680721C90288432969C90078
:1074D0000843E06000F03AF8E168094A0906090F3C
:1074E000515CC8400749086007480068FFF7C0FBC7
:1074F000F8BD000000200240881300000010024088
:1075000062C7000878010020700100200448054986
:107510000068C968044A4905490F515CC840704772
:1075200078010020001002407BC70008044805498C
:107530000068C968044A8904490F515CC840704713
:1075400078010020001002407BC7000870B51A4A7D
:10755000D3681A490C2018408D0004280CD04E0026
:10756000082810D00C2810D050680004410F0120CA
:10757000C003491C884070BD1068C00601D508468C
:1075800070BD284670BD304670BD98020C4C000F8F
:10759000205C1B029C0FD368641CDB0301D53146C1
:1075A00003E01268D20600D4294603F0CCF8224644
:1075B0000023FDF7B3FD70BD0010024000093D003F
:1075C00072C70008FEB505007ED0FE4CE7680C20AF
:1075D000E66807400120000406402878C00747D02D
:1075E000082F05D00C2F0AD101200004864206D1B5
:1075F000206880033CD568680028E5D038E0012089
:1076000069680004814203D121680143216011E0CF
:10761000052301221B0492049942216802D11143DF
:107620002160F1E7814321602168014000912068D9
:1076300090432060686800280DD0FFF7F7FA0090AB
:1076400005E0FFF7F3FA0099401A64287BD8206818
:107650008003F6D50CE0FFF7E9FA009005E0FFF7AC
:10766000E5FA0099401A6428F0D820688003F6D41F
:107670002878800756D50923E868042F0DD00C2FF1
:1076800001D1002E09D000283CD021689943014344
:107690002160FFF7CBFA064628E02168490701D5AB
:1076A000002891D061681F22120291432A691202B8
:1076B000114361602168994301432160FFF746FF50
:1076C000E16809060A0F00E08BE1BF49895CC84008
:1076D000BE490860BE480068FFF7CAFA002873D1A7
:1076E00020E0FFF7A3FA801B0228AFD820684007EC
:1076F000F7D560681F2109028843296909020843F8
:1077000060600FE02068400840002060FFF78EFABC
:10771000064604E0FFF78AFA801B022896D8206804
:107720004007F7D42878C00660D5002F0CD0A86990
:1077300000284AD02068FF21013108432060FFF76C
:1077400075FA06462EE0C1E02068800502D5A869DA
:107750000028A6D06068072149038843296A0843A6
:1077600060606068297F0002000A090608436060C3
:10777000286A410B0120C003491C8840E1680906C2
:107780000A0F9149895CC840904908609048006898
:10779000FFF76EFA002817D128E0FFF747FA801BA1
:1077A0000228A2D820688005F7D560680721490320
:1077B0008843296A084360606068297F0002000AE4
:1077C00009060843606011E0E2E02168FF20013013
:1077D00081432160FFF72AFA064604E0FFF726FA04
:1077E000801B022872D820688005F7D42878794E4B
:1077F000000724D568690028306910D001210843AA
:107800003061FFF713FA009005E0FFF70FFA0099D7
:10781000401A02285AD830698007F6D50FE0400890
:1078200040003061FFF702FA009005E0FFF7FEF933
:107830000099401A022849D830698007F6D4287880
:10784000400766D500200290A06BC00006D4A06B54
:10785000012109070843A063012002905E480168E6
:10786000C90511D40168821511430160FFF7DEF9E3
:10787000009005E0FFF7DAF90099401A642825D84E
:1078800055480068C005F5D5FF20AA68013082423E
:1078900003D131690143316111E001218902002ADC
:1078A00007D005231B029A4203D132690A43326191
:1078B000EFE7326982433261306988433061A868FA
:1078C000002810D0FFF7B2F9009008E05FE0FFF762
:1078D000ADF901460098091A4048814257D83069ED
:1078E0008005F4D50DE0FFF7A1F9009006E0FFF761
:1078F0009DF90099411A3948814248D8306980057C
:10790000F5D40298002804D0A06B01210907884310
:10791000A063686A002866D00C2F3ED00126360688
:107920000228206805D0B0432060FFF77FF90546A4
:107930002FE0B0432060FFF779F9074604E0FFF736
:1079400075F9C01B022822D820688001F7D4E96AA3
:10795000A86AE2680843296BFD231B049A4311437C
:107960000843E060206830432060FFF75FF9054678
:1079700004E0FFF75BF9401B022808D8206880016B
:10798000F7D530E0FFF752F9401B022801D9032058
:10799000FEBD20688001F5D425E00128F8D0E0681C
:1079A00001210904AA6A014091421AD10F218904D8
:1079B000EA6A0140914214D1032189050840296BEC
:1079C00088420DE00010024062C7000878010020E4
:1079D0007001002040100240007000408813000039
:1079E00001D00120FEBD0020FEBDF8B504000ED080
:1079F000FF27606A0537002500280AD025616561E8
:107A000026464036A562707C002807D00AE0012097
:107A1000F8BD6068B842F3D0E561F1E735742046FF
:107A200000F03EF8022171742068026840239A43F6
:107A300002602123A26860689B021A40384010430C
:107A4000E3688A021340184323690B40217D1843E1
:107A5000C907C90F0843A169931019400843E16998
:107A6000382319400843216A802319400843A16A3A
:107A700093001940084321680860A0690421000CA4
:107A80000840616A10231940084321684860206853
:107A9000C1699143C1616565012070740020F8BD22
:107AA00010B586B0044614216846FDF780FB1049E6
:107AB0002068884219D10F48416B821411434163F9
:107AC000C16A01221143C162C06A002110400590C1
:107AD000E020009002200190032003900291049185
:107AE000052069460007FEF7D1FF06B010BD000073
:107AF0000030014000100240094910B5401E884284
:107B000001D9012010BD074C60610321081F02F05C
:107B100055FE0020A06107202061002010BD00005C
:107B2000FFFFFF0000E000E0F0B502462032137EC8
:107B3000012B1ED001251576022353760668746842
:107B4000B3687027BC430F68274377600068AC07B1
:107B5000A04205D0084CA04202D0084CA04204D15B
:107B600080244968A343194381605576002010762C
:107B7000F0BD0220F0BD00000008014000140140EB
:107B800070B5050005D02C462034607E002802D058
:107B900006E0012070BD00202076284600F010F895
:107BA00002206076291D286802F020F80120A077C5
:107BB000A076E076207760776076002070BD0000C8
:107BC000006801218907884204D10348816B0122A2
:107BD000114381637047000000100240F8B505466C
:107BE00004462035287E012817D001262E76022053
:107BF0006876226890687727FF23B8431B02984372
:107C000090600A68502A31D00EDC202A4BD006DC66
:107C1000002A48D0102A3AD145E00220F8BD302A87
:107C200041D0402A33D136E0602A27D0702A12D0C2
:107C300001200003121A2AD0824228D1CB684A6858
:107C40008968206802F00BF820688168012292039D
:107C5000114381601BE0CB684A688968206801F0A5
:107C6000FEFF216888683843886010E0CA68496868
:107C7000206802F06EF85021206806E0CA68496862
:107C8000206802F077F86021206801F0F3FF6E763B
:107C900000202876F8BDCA684968206802F059F8C3
:107CA00040212068F1E711462068EEE710B586B064
:107CB000044614216846FDF77AFA012120688907F5
:107CC000884212D10A49CA6A02200243CA62C96ABA
:107CD0000190014005914102009100210291039120
:107CE000049069460348FEF7D1FE06B010BD0000BF
:107CF0000010024000040050F8B506460446203645
:107D0000307E0D4601280BD0012008273076002A4E
:107D100008D0042A16D0082A2AD00C2A4DD137E0E0
:107D20000220F8BD206801F0ADFF20688169394369
:107D300081612068816904229143816120688169A1
:107D4000EA6812E0206801F0B5FF2068816901222D
:107D5000D2021143816120688269012189028A432C
:107D6000826120688169EA6812021143816124E01E
:107D7000206801F0B8FF2068C1693943C1612068FB
:107D8000C16904229143C1612068C169EA6812E0B7
:107D9000206801F0C3FF2068C1690122D2021143AB
:107DA000C1612068C269012189028A43C2612068D9
:107DB000C169EA6812021143C16100203076F8BD42
:107DC00070B5050005D02C462034607E002802D016
:107DD00006E0012070BD00202076284600F00FF854
:107DE00002206076291D286801F000FF0120A0779D
:107DF000A076E076207760776076002070BD7047CF
:107E000070B505462C4602202034002908D00429EC
:107E10000BD008290ED0627F012A10D0012070BD3E
:107E2000A27E012AFAD1A0760AE0E27E012AF5D1EB
:107E3000E07605E0227F012AF0D1207700E060772C
:107E40000122286801F0FEFE012228689207012124
:107E5000904205D0074A904202D0074A904204D18E
:107E600082685207520F062A02D002680A43026053
:107E7000002070BD000801400014014070B50446A8
:107E80000D460068002201F0DDFE2068016A0C4A00
:107E9000114203D1016849084900016001202034E2
:107EA000002D06D0042D06D0082D06D060770020C6
:107EB00070BDA076FBE7E076F9E72077F7E70000F2
:107EC000111100007047704770470000F8B5026854
:107ED0000446D06911689668814B05461D402023F1
:107EE000002D6CD0F7077F4DFF0FBC460D402F4390
:107EF00079D02546C7078035002F06D0CF0504D599
:107F0000012717622A683A432A60820708D5F207D8
:107F100006D0276802223A622A6804273A432A6078
:107F2000420708D5F20706D02668042232622A6882
:107F3000022632432A6002070AD50A461A406646DC
:107F4000324305D02668082232622E6816432E601E
:107F5000020508D54A0106D501222668D2023262FE
:107F60002A681A432A602A68002A30D0800606D57B
:107F7000880604D5616E002901D02046884728680C
:107F800021688968490602D42821084225D0204664
:107F900002F01FF920688168490619D582684021DE
:107FA0008A438260206F002812D04F498163206F7E
:107FB000FEF7D2FB00280AD0206F816B06E0850611
:107FC00011D58D060FD5616E77E020468847F8BD44
:107FD0002046FFF779FFF8BD05E02046FFF774FF64
:107FE00000202860F7E7256E012D56D1C50654D52F
:107FF000CD0652D5102616622068816825464906AE
:10800000403500292ADA226F116849680904090CF1
:10801000E1D02F8B8F42DED9698311680968890608
:1080200017D40168320191430160206881684908D2
:108030004900816020688168402291438160E36744
:108040000020206620680168B1430160206FFEF7C0
:1080500061FB288B698B401A81B21AE0298B6A8BED
:10806000891A6A8B89B2002AB5D00029B3D0026878
:10807000FF252135AA430260206882685208520019
:108080008260E36700202066606620680268B24371
:1080900002602046FFF716FF9DE7C50208D575026E
:1080A00006D50120000510622046FFF70CFF92E77D
:1080B000050605D50D0603D5A16E002985D18AE7F1
:1080C000400688D5480686D5116820464024A1433D
:1080D000116083670021816600F043F97BE70000AF
:1080E0000F08000020010004F9A0000810B50400EA
:1080F00003D0A06F002802D007E0012010BD0021AE
:1081000074200155204600F027F82420A06720683D
:108110000168490849000160204602F0ADF80128D5
:10812000ECD0606A002802D0204601F0C5FE20682D
:1081300041680922D20291434160206881682A2265
:10814000914381602068016801221143016020464B
:1081500001F018FF10BD0000F0B587B006461421ED
:108160006846FDF724F82C493068884251D12B48E5
:10817000416B0122920311434163C16A0122114301
:10818000C162C06A002510400590032040020090A3
:108190000220032701A9A1C10420049005206946FB
:1081A0000007FEF773FC1F4C1D48A560E56081C405
:1081B0008027E560A7602020256160610002A06142
:1081C0001848083CFEF742FB002801D0FDF71CFED2
:1081D0003467A662144C12482146143820600320EC
:1081E000606010200831A1C16561A561E56120468C
:1081F0002562FEF72BFB002801D0FDF705FEF46693
:10820000002201211B20A662FEF7A2FF1B20FEF721
:1082100093FF07B0F0BD000000380140001002409D
:1082200030000240301700207817002070B5C36F6F
:10823000202B27D100290BD0002A09D001248368E4
:108240002403A34206D10369002B03D1CB0701D03D
:10825000012070BD034660331C7D012C12D0012427
:108260001C7500230366084C0368A34207D05C68B2
:10827000240204D51C680125AD062C431C6002F0C5
:10828000FBF870BD022070BD004800407047704789
:10829000FFB50446806F83B017460D4620285ED197
:1082A000002D0AD0002F08D0A168C001814207D15B
:1082B0002069002804D1E80702D0012007B0F0BDF2
:1082C000204660300090007D012848D000980121B0
:1082D00001750020802108512120A067FEF7A6FC2F
:1082E000264640360190378277820120A16800033C
:1082F000814202D12069002805D02F46002500992F
:108300000020087511E00027F9E7002280212046AF
:1083100002F0F8F8002815D1002F15D02168387820
:1083200088627F1C708A401E7082708A019B0028C0
:1083300006980090E9D100224021204602F0E2F8A0
:10834000002808D00320B9E728882168C005C00D9F
:108350008862AD1CE6E72020A0670020AEE702207F
:10836000ACE77047034D044C04A002F0CBF9E56084
:10837000FAE700000400FA0500ED00E048617264CD
:108380004661756C745F48616E646C65722E0D0A8F
:108390000000000030B585B014216846FCF707FFE7
:1083A0001148418B002901D10221418388B2012863
:1083B00007D0022803D100F003FCFDF747FC05B00D
:1083C00030BD0122094D940221462846FEF727FCC4
:1083D00000210120029103910190009469462846F2
:1083E000FEF754FBEBE700002401002000040050DE
:1083F00010B505242407002204212046FEF70FFCB7
:10840000002208212046FEF70AFC0A2002F0DFFBCA
:10841000012204212046FEF702FC0A2002F0D7FBCD
:10842000002204212046FEF7FAFB10BD10B50524FA
:108430002407002204212046FEF7F1FB0122082137
:108440002046FEF7ECFB0A2002F0C1FB01220421CA
:108450002046FEF7E4FB0A2002F0B9FB00220421CB
:108460002046FEF7DCFB10BDF8B5002405260746C4
:1084700025463607002204213046FEF7D0FB0A20AD
:1084800002F0A5FB012204213046FEF7C8FB60067E
:10849000040E08213046FEF7B5FB002801D0641C0D
:1084A000E4B2052002F093FB6D1CEDB2082DE1D380
:1084B000002F03D0FFF79CFF2046F8BDFFF7B6FF63
:1084C000FAE770B505260546360700220421304636
:1084D000FEF7A5FB0024E80901D0012200E00022FC
:1084E00008213046FEF79BFB6806050E0A2002F0C5
:1084F0006EFB012204213046FEF791FB0A2002F0B8
:1085000066FB002204213046FEF789FB0A2002F0B8
:108510005EFB641CE4B2082CDDD370BD10B50524ED
:108520002407012208212046FEF779FB01220421BD
:108530002046FEF774FB002208212046FEF76FFB61
:108540000A2002F044FB002204212046FEF767FBCC
:1085500010BD10B505242407002204212046FEF793
:108560005EFB002208212046FEF759FB0A2002F09C
:108570002EFB012204212046FEF751FB0122082197
:108580002046FEF74CFB0A2002F021FB10BD70B51F
:1085900005252D070024012208212846FEF73FFB70
:1085A000062002F014FB012204212846FEF737FBC7
:1085B000062002F00CFB07E0641CE4B2FA2C03D99D
:1085C000FFF7C7FF012070BD08212846FEF71AFB00
:1085D0000028F1D1002204212846FEF720FB0020CC
:1085E00070BD0000F8B501F0FFFC01F039FD5848FE
:1085F0000068C069FDF7F8FC564C5749A082898F86
:10860000564E0025002931D0A26A730354499A427C
:1086100002DB02220A7000E00D700A780121890253
:10862000002A05D0012A0ED0022A10D0032A1DD11B
:10863000608B01282BD0022818D1454808214038EA
:10864000FFF71CFC12E0FF22F5329042F0D2608B63
:1086500001281AD0022804D008E03046FEF7DFFADD
:1086600004E03B4808214038FFF7CAFB0121C9025A
:108670003046FEF7C7FA0127FF0300282AD0394801
:108680000560E079002804D007E00022E5E7012238
:10869000E3E70120E07101F097FF2078632806D915
:1086A000002208213046FEF7BAFA012205E0012235
:1086B00008213046FEF7B3FA0022052039460007AC
:1086C000FEF7ADFA244C284E4034A08C274F0128E9
:1086D00003D01CE0E5710022EAE7254869460880DE
:1086E00072B680212348FDF7A7FB002804D00222A0
:1086F00069462048FDF744FC62B61FA002F002F86C
:10870000A58403F041FF642002F05AFAFE60608CF9
:10871000012808D110486584058003F035FF6420E6
:1087200002F04EFAFE60208C012806D1258403F069
:108730002BFF642002F044FAFE600748124A0188C9
:10874000914202D1C088002800D1FE60F8BD00002F
:10875000AC16002024010020DC0D00200004005095
:1087600081000020680100200400FA0500ED00E00F
:10877000AAAA0000384A0008BDF8C8EBC9FDBCB67B
:10878000C4A3CABD0D0A0000AA55000008B53721D0
:10879000202000F06EF80321212000F06AF840212B
:1087A000222000F066F80821232000F062F8AA21B8
:1087B000302000F05EF80A48008FC1B2322000F08D
:1087C00058F80221332000F054F85F21202000F0F7
:1087D00050F8684600F006F80A2002F0F8F908BDE3
:1087E000DC0D002010B501460F2000F021F8002814
:1087F00000D0012010BD10B50446FFF78FFE3220D7
:10880000FFF75FFEFFF7C3FEE0B2FFF75AFEFFF788
:10881000BEFEFFF783FE3320FFF753FEFFF7B7FEE0
:108820000020FFF721FE0446FFF793FE204610BD0F
:1088300010B50C46FFF7DFFF2070012010BD70B5AA
:108840000D460446FFF76AFE3220FFF73AFEFFF7B7
:108850009EFEE0B2FFF735FEFFF799FE2846FFF7D0
:1088600030FEFFF794FEFFF774FE0A2002F0AFF926
:1088700070BD10B5FFF7E3FF012010BD10B5024831
:10888000FEF719FB10BD0000E4150020FEB50446FC
:10889000002772B6334A01688B1804D13248C76882
:1088A00003208004074088680190C86800904869E8
:1088B0008E69002B08D12C4940398B6ACD042B439B
:1088C0008B628B6AAB438B62014631433CD02549B6
:1088D0002368CB4205D12449CA6803239B049A43E9
:1088E000CA6025462035002810D021680A69012376
:1088F0001A430A61216848610821204600F036F8D1
:10890000032800D1A873216808204860002E10D0E9
:1089100020680169012211430161206886611021EC
:10892000204600F023F8032800D1A8732168102006
:1089300048600C482168C14206D10B48C168032237
:10894000920491433943C160206801694908490094
:10895000016121680198886021680098C86062B64A
:10896000FEBD00000084FFBF4010024070B5064607
:108970000B480D46002409490068FCF7B9FB7D212E
:10898000C90048433168401E00D103240B682A46C1
:108990009A4301D00028F6D1204670BD204E000039
:1089A000780100201CB5002116480091144A01915D
:1089B0000260C16312054260816007228263012266
:1089C00002610246C16020321170FF235170C23330
:1089D00043628162117301638161042241634261D8
:1089E000C161FDF7FDFC08480090801301906946C5
:1089F0000448FDF7A5FC00210248FDF74BFC1CBD17
:108A000000240140881500200200000408B5084831
:108A1000016B012211430163006B012110400090A2
:108A200000220A20FEF794FB0A20FEF785FB08BD12
:108A300000100240F0B587B014216846FCF7B7FB80
:108A40004748C26A04210A43C262C26A0A400592C8
:108A5000C16A80263143C162C16A31400591C16A51
:108A600001242143C162C16A21400591C16A0225E6
:108A70002943C162C06A22462840059005201C2176
:108A80000007FEF7CCF8012236493748FEF7C7F851
:108A9000002236493448FEF7C2F891210520002211
:108AA00009020007FEF7BBF83148019000270520B6
:108AB0006946029700940007FDF7E8FF0C2000903C
:108AC00011200190032003900520029769460007BA
:108AD000FDF7DCFF10206A46039591C20520694628
:108AE0000007FDF7D3FF1120019002976946039715
:108AF00000941D48FDF7CAFF1E4801906946009585
:108B000002941948FDF7C2FFE00200906946019700
:108B100002951548FDF7BAFF1748694691C16946A5
:108B200011480397FDF7B2FF91200002694691C1F9
:108B30000520694600070397FDF7A8FF69460A4824
:108B4000019700960294FDF7A1FF00220121052064
:108B5000FEF7FEFA0520FEF7EFFA07B0F0BD0000C1
:108B60000010024001020000000400500830000024
:108B700000001110000021100832000010B50F4C49
:108B80000D482060FF20053060600020A060E0609C
:108B900020616061E0610121206249026062A1619F
:108BA000A0620720E0622046FEF71FFF20680168F0
:108BB00040221143016010BD003001401416002016
:108BC00010B58AB000240494059406940794089480
:108BD0000121184809940094019402948907039490
:108BE0000160092184604160046113494461C160EE
:108BF000FEF7C6FF01200003049004A90D48FEF70C
:108C0000EDFF0C48FFF7DCF8089408A9094809941F
:108C1000FEF78AFF60200090084801900294082225
:108C2000694603940348FFF767F80248FFF73EF8E8
:108C30000AB010BD6C16002093040000570200001B
:108C400000B585B014216846FCF7B1FA0E480D490D
:108C50000160E1214902416000218160C160016140
:108C600081610C22C16142610162302141620121B6
:108C7000090381634900C163FFF738FA01F09EFCE4
:108C800005B000BD00380140AC1600207047000060
:108C9000F0B585B00A2002F0E5FC7D20C00002F0AE
:108CA000FBFCFF4C0025A570FE48A065607B0C28EE
:108CB00001D30B206073FC48E570FC4E00783071E6
:108CC000FB49A079097840000843E17C890008430A
:108CD000F071606BF070010A3172401C6063607962
:108CE000B07442003046F3491330FCF747FA60791C
:108CF000F04982004000801962311330121DFCF7E8
:108D00003DFA3020205E002803D0EB49098A08187C
:108D10002086607906214843E149E44E20318219DA
:108D20000B7CD3754B7C137606227272E34A1C309F
:108D30001278B272628C32733246133A0B79137521
:108D4000497951750022314602F076FD607906219D
:108D5000484300211C3002F081FD022002F0D2FCC9
:108D6000F571E573A57201202073E572D448FEF712
:108D70007DF920850646E5706079FCF7DFFCD14A75
:108D8000D14BFCF7BFFB01F0B7FE012300229B078C
:108D9000FCF706FBFCF732FD0006C10C881980B217
:108DA0000121C9036085884201D3401A6085C74804
:108DB00060642079401C2071C148FEF757F9B84E15
:108DC000E0844036F6E1BE48FEF750F9E084C04F3B
:108DD0000BE0BB48FEF74AF980B2E084618D88421F
:108DE00003D3BC4A8918884206D300210F2002F021
:108DF000B9FB3842A063ECD0A06B411C21D04004E9
:108E00007ED58122D20100210F2002F0EAFC7D20D4
:108E1000C00002F041FC002002F0F3FB0021102012
:108E200002F0A0FB4106A348490E274600227E38E7
:108E3000616502F0CDFB9F487E38417A0729C1D198
:108E400001E001F0DDFC0222A349401DFCF7BAF964
:108E50000028B7D102F053FD7966386602F03CFD78
:108E6000F966B866F8786946401CF870914885380C
:108E7000027A0A70407A487008880090B98C88425B
:108E80007ED18A48954F8C30C08E8849388084487E
:108E90008C31098F01848A48FEF7E8F8E08402F0FB
:108EA00073FAFF22A16E5204E06E00238918584124
:108EB0000206080A1043410849000190080E090201
:108EC000216760677948636E0A30226E02F0ECFC1D
:108ED0006079E36E81007548A26E0818163002F0C2
:108EE000E3FC7248636F1230226F02F0DDFC6F48C2
:108EF00008214172A17CCA300090002915D000E001
:108F00004BE1022274491138FCF75CF900280CD1BE
:108F100001206649E073C871606D1638C2B26548B9
:108F200022749E300099FCF729F902226A490098C0
:108F3000FCF748F9002827D15E4855211A380170FE
:108F4000AA2141700E2181701221C1701022001DD2
:108F50000099FCF713F9574851492638408A48834D
:108F6000218B814210D02083524812211838FCF7FF
:108F700091FE5049E0832639088416214D4800E0CF
:108F8000D8E01A3801F046F960790022800047499C
:108F90001C3002F051FC6079002180001C3002F08E
:108FA0005DFC019802F057FB012002F0ABFB207240
:108FB00002214B48FDF726FE00286FD000203C49D7
:108FC0003C4B0870394862338C30428E3280818E3F
:108FD0007180206C606418601846E038C37C180704
:108FE000000F032800D060741809A07425710120B7
:108FF000A072B280F180E072208C3A49FF30C33019
:1090000080B2208488420BD9494240182084388895
:109010007D21401C80B2C9003880884200D33D8049
:109020003E887D20C000218C70434018A0640390CE
:109030002D48302107782D48A77300884843FCF756
:1090400062FB00900A2031464143608C302202903E
:109050005043081AFCF74CFB0099FCF756F97F21A6
:10906000C905FCF7BCF8FCF790FB80B21E497F1ED7
:109070000880B84201D10120E072A6851620205E4A
:10908000FCF748FB06460F46E08CFCF757FB184AF6
:10909000184BFCF737FA019100902DE041E00000F9
:1090A000700000203F420F002401002050120020D9
:1090B00064010020821300201C0E002034010020D7
:1090C000E4150020B81E85EB51B8CE3FA086010004
:1090D00000D02724983A00004801002060010020B9
:1090E00000040050E703000040010020440100207C
:1090F000F853E3A59B843E400398FCF70BFB019BD0
:10910000009AFCF7F1F932463B46FCF749F9FCF7C7
:1091100051FBE064029800F0A1FC207A002802D004
:1091200051E001204BE700210F2002F01BFA00065E
:10913000F9D548E0FCF740FF4C4A032111544C4953
:1091400080004A8E3280898E71804849484A603951
:1091500001904118928F0A8044493A6C3039411885
:109160004A604349FB6E8C3940181630BA6E02F0E3
:109170009BFBB96D386C884200DAB8653B49019AAF
:1091800060398958814215DD002913D0002811DD8E
:109190000098B884022038700CE03A4600210F2075
:1091A00002F01FFB6079E178401C814202D0002070
:1091B00002F027FAE18C608D814200D203E62D4A4D
:1091C00080188142FAD8A07A012801D00220A0722A
:1091D00002F0DAF8284A00210F2002F002FB207981
:1091E000002806D025490A2209885143814200D22D
:1091F0002570E07B00281ED01C490C310B78487884
:109200008A78022B17D110280CD0C82813D21C4BF7
:10921000C91C1818FBF7B2FF03F0B6F9642001F07F
:10922000CFFC0EE6174D28684000000E03D1C87829
:10923000FCF769FA28600D4D0020923D2E462278F9
:109240006379183607E041006F5A715A8F4200D097
:109250000222401CC0B29842F5D32270064A002177
:1092600080320F2002F0BDFA05B0F0BD14140020CA
:10927000DC120020983A000000D02724340100209E
:10928000DC0D00204C01002070470000F0B58DB0CF
:10929000002005900A2002F0E5F97D20C00002F0D0
:1092A000FBF9BE4800218170426BBD4C521C4263E9
:1092B0000175214613310991BA49079121465A3166
:1092C000029126466D393136B74F20300691039012
:1092D000B24D0F21B548697100782071B44AA87960
:1092E000127840001043EA7C92001043E071A88E8F
:1092F000E070000A2072A17429461E228431099868
:10930000FBF73CFF40223046AA49FBF737FF07989E
:10931000298E008A40182886039902980A7CC27414
:10932000497C017509206072A3480078A072688C9E
:109330002073287D410028468430091806980A7851
:1093400002754978417576200022954902F074FA39
:1093500068790621484300211C3002F07FFA022080
:1093600002F0D0F900210F2002F0FCF83842A86387
:10937000F8D0A86B411C18D040047CD58122D201C2
:1093800000210F2002F02DFA0021102002F0EAF84F
:1093900041068348490E0022B43002F019F9804892
:1093A000B430417A022902D0D1E001F029FA022238
:1093B0008249401DFBF706FF0028F5D177480222BD
:1093C000007D41007548843009187548B530FBF7B9
:1093D000F9FE0028E8D102F092FA704D696628661D
:1093E00002F07AFAE966A8660598002846D10120BD
:1093F00005906B48724D8C30C08E69492880674853
:109400008C31098F01846F48FDF730FE63496E4A45
:10941000C884088CFF30C33080B2088490420CD9D5
:109420005242801808842888674A401C80B20B3258
:109430002880904201D30020288028887D22D200F5
:109440000B8C4243D2188A64604A1288D3B2944685
:1094500002460A3A12B28B73CA85002A03DA7D25C6
:10946000ED005219CA855B1E9C4501D10122CA72CA
:109470008885488C00E08BE000F0F0FA48486946A7
:109480008C30428E0A80808E488045490422B53156
:10949000C81FFF38FBF772FE4048464A007D00991E
:1094A000800011503D48FF23816EC06E5B04002296
:1094B000C918504100060D0A0543284602F0CBF8B2
:1094C00068084000020E0102344800254267016727
:1094D000436E026E3248483802F0E6F92F48C36EF8
:1094E000826E2F48443802F0DFF92C48436F026F38
:1094F0002B48403802F0D8F92949002252393C2043
:1095000002F09AF900213C2002F0A8F9012002F0B3
:10951000F9F82249087208468078401C88700121B9
:109520000520C9030007FCF75BFD1C48007A0028F2
:1095300005D100210F2002F015F80006F9D5802290
:1095400000210F2002F04DF914494D7002E013493B
:10955000012048701148017D491CC9B201750F29CD
:1095600000D2B5E60598002810D10C481849428C65
:10957000002A02D00B889A4201D9098841841549F2
:10958000408C0988401E4843134908800DB0F0BD47
:10959000124A00210F2002F024F9D8E770000020C1
:1095A000501200201C0E002000D02724240100208F
:1095B00064010020701400203401002048010020C4
:1095C00060010020E4150020E703000040010020B6
:1095D000300100202E0100202C01002000902724C3
:1095E000F8B532493048086002F072FA304800F0AD
:1095F000F5F9304CE0822E48801C00F0EFF9208312
:109600002B48001D00F0EAF960832C482A4941806C
:10961000014640310A792A4F1206120E627006D1B5
:10962000C7800122C2870A224287002282870289DC
:109630000A82244AC18E1170C18F6171818FA1711C
:10964000817AE1708588052165626181C68830462E
:10965000FBF74EFDA08101462846FBF749FD880037
:10966000081885B2164825816843FCF767F8164A42
:10967000164BFBF7AFFFFCF7C1F8E081658231467E
:109680003846FBF735FD20820146C820FBF730FD48
:1096900020840120A083FCF7A7FCA082E2890C496A
:1096A0000C48FDF7E7FCF8BDF5A5000868000020B0
:1096B000004F0008240100201B020000DC0D0020E8
:1096C000E803000018000020F853E3A59B843E4007
:1096D000FF7F0000E4150020F0B59A4D85B0012011
:1096E0002880994FC820994C3880E079401CE0715F
:1096F000C00706D0608C411E6184022801D2C820B8
:109700006084608C00F0AAF90A2001F0ABFF7D2094
:10971000C00001F0C1FF02218D48FDF773FA002857
:109720003FD000208B49800009788C4E49000843C7
:10973000894909780843B072102070728848C1883E
:109740007D20C000FBF7D4FC707386488449007804
:10975000B07330460B308A780270C9784170804906
:10976000421C20310B7ED370497E11717C49D01C84
:1097700022310B7E5371497E9171794940310A7CC7
:109780000271497C417100223146172002F054F8E1
:109790000021172002F062F8022001F0B3FF724EA0
:1097A00003E00120BEE7FEF71DFF00210F2001F0BE
:1097B000D9FE3042A063F6D0A06B411C7ED040049D
:1097C0007DD58122D20100210F2002F00AF800216C
:1097D000102001F0C7FE41066048490E0022B43057
:1097E000616501F0F5FE5D4EB436707A112866D1E0
:1097F00002225E49701DFBF7E5FC00285FD1F01FD7
:10980000027A69460A70407A4870B17A2980C82085
:10981000FBF76EFC3880307B60843046544D28382E
:10982000C08E2880314649482839098F0184514823
:10983000FDF71CFC80B2E0840390208C4E49FF3081
:10984000C33080B2208488420CD949424018208419
:1098500028884949401C80B20B312880884201D3B6
:10986000002028802D887D20C000218C684340186E
:10987000A06402904148067828460A3800B2A673D0
:10988000E085002803DA7D21C9004018E08538888A
:1098900030214843FBF737FF07462E20205EFBF7B9
:1098A00027FF3946FBF731FD7F21C905FBF797FC00
:1098B000FBF76BFF314980B2088001E03FE03CE0FC
:1098C000761EB04201D10120E072A5851620205EEF
:1098D000FBF720FF074601910398FBF72FFF284A6B
:1098E000284BFBF70FFE05460E460298FBF712FFCA
:1098F0002A463346FBF7F8FD3A46019BFBF750FD3D
:10990000FBF758FFE06468460088A08413481349B9
:10991000B430807CC7316071420008460D466B3020
:10992000FBF72CFC6079294642001748FBF726FC20
:10993000608CFF2801D00320207005B0F0BD00F03E
:109940005FFF00003401002044010020700000206F
:1099500000040050290100202A010020501200209C
:10996000DC0D00201800002000D027244801002032
:1099700060010020E4150020E70300004001002002
:10998000F853E3A59B843E409A13002070B586B03F
:1099900014216846FBF70BFC01250F4EED03002256
:1099A00029463046FDF73BF901200024019002943E
:1099B0006946009503943046FDF768F8032001904E
:1099C00002946946009503943046FDF75FF8022043
:1099D00001F0F6F806B070BD000400500088704732
:1099E00070470000F8B5044600206A461080194D03
:1099F00055222A70AA226A700322AA70661DEE7090
:109A00002A716971144A49008918AC712246E81D0F
:109A1000FBF7B4FB002007E029186A468978128812
:109A200089186A461180401CB042F5DB611DA81CF4
:109A3000FCF730F901466846018029190078C871A1
:109A400068464078087221460931024800F0E2FB7E
:109A5000F8BD000024150020DC0D002010B51B4CC3
:109A6000228A01E0891AA183A18B9142FAD2228C29
:109A70008BB253431B18E383132902D14A431018B6
:109A8000E083E08B3021484364216430484310492F
:109A900060630968401A4B21090140182063FBF7F5
:109AA00039FE0C4A0C4BFBF795FDFBF783FE0B4987
:109AB000E062884202DD4A428018E062002801DA52
:109AC0004018E06206490968486110BD2401002081
:109AD000BC000020F853E3A59B843E40FF7F0000BC
:109AE000E4150020034A1168382389B299430143E1
:109AF000116070470030014010B5FDF79DF810BDB2
:109B000010B59AB034216846FBF751FB14210DA81B
:109B1000FBF74DFB1C2112A8FBF749FB1B48016812
:109B20000324E402A143C21489180160FDF71CFB61
:109B300017480169A143016106200090FF20013010
:109B4000029001200390102004900220099040040C
:109B50000B90000100240C900A946846FDF732FD3A
:109B60000F200D9003200E900F941094012111945A
:109B70000DA8FDF7FDFB81201290032080041890B2
:109B8000149412A8FDF742FB1AB010BD00700040FB
:109B90004010024010480168821511430160C168FD
:109BA0000E4A1140C16001680D4A11400160816890
:109BB00049084900816001680122920491430160D3
:109BC000C168FD2212049143C16000210161064970
:109BD0000448886070470000001002400C40FF8875
:109BE000F6FFF6FE0050000800ED00E070B50268D8
:109BF00001239B07114C124D984203D0A04201D083
:109C0000A84203D17026B2434E683243984203D033
:109C1000A04201D0A84204D103231B029A43CB687F
:109C20001A4380239A430B691A4302608A68C2620E
:109C3000096881620121416170BD00000008014096
:109C40000014014010B5CB06DB0E0121046A9940D7
:109C50008C430462016A9A401143016210BD30B521
:109C60008468FF252D021B021343AC430B4323439F
:109C7000836030BD826870239A430A4307210A43F8
:109C80008260704730B5026A520852000262026A6E
:109C9000456883697024A3439C080B68A400234390
:109CA0000224A2438C684560144383614968416380
:109CB000046230BD30B5026A10239A430262036A1F
:109CC0004568826973242402A2430C682402144369
:109CD000202293438A68456012011A4384614968CF
:109CE0008163026230BD30B5026AFF2301339A43BB
:109CF0000262026A4568C3697024A3439C080B682A
:109D0000A400234301246402A2438C68456024021A
:109D10001443C3614968C163046230BD30B5026A4F
:109D200001231B039A430262036A4568C2697324D4
:109D30002402A2430C6824021443012252039343D9
:109D40008A68456012031A43C4614968016402626B
:109D500030BD30B5036A046A640864000462846933
:109D6000F025AC43120122430A24A3430B43826132
:109D7000036230BD30B5036A1024A34303628469D3
:109D8000036A0F252D031203AC432243A024A343EF
:109D9000090119438261016230BD0000F8B5102647
:109DA00005252D07AE62AF20800000F010FFFCF704
:109DB000B1F9364834490068FBF76AFAFBF7CCFC86
:109DC000334C2086AE6101F0E1FB324F324EE0654C
:109DD0000EE001F0DBFBE065FEF704FCE06B411CEC
:109DE000E163142804D92DA000F08CFC2F48C76033
:109DF000E06DB042EDD10026E66320780127FF0335
:109E0000030000F0B8FC05040C192D3032000122CB
:109E100039462846FCF703FFFFF75EFC06E0012207
:109E200039462846FCF7FBFEFFF730FA0022394698
:109E30002846FCF7F4FE18E0607A0122401E6072AA
:109E400039462846FCF7EBFEFCF7EAF800223946D3
:109E50002846FCF7E4FE607A002806D1267004E06C
:109E6000FEF716FF01E0FFF711FA02211048FCF798
:109E7000C9FE002805D000200E49087001F06CFAD8
:109E8000F8BD0120F8E700000000C84200000020F3
:109E9000700000200400FA053001CADE4457204952
:109EA00044204552524F522E0D0A000000ED00E0B2
:109EB000000400506401002010B5818CC90707D050
:109EC00001684A6801235B049A43836A1A434A6023
:109ED000818C890707D501684A6801231B049A43CE
:109EE000C36A1A434A60818C490707D501684A68EA
:109EF00001239B049A43036B1A434A60818C090730
:109F000007D501684A680123DB039A43436B1A4370
:109F10004A60818CC90607D50268916801231B033A
:109F20009943836B19439160818C890607D5016839
:109F30008A6801235B039A43C36B1A438A60818C4E
:109F4000490612D503685A6801210905046C8A4341
:109F500022435A60026C8A4207D102685168032387
:109F60005B059943436C19435160818C090607D501
:109F700001684A680123DB04806C9A4302434A600B
:109F800010BD0000F8B50446002680300660FCF7DE
:109F90004DFE054620680068124F000709D50121D3
:109FA0002B46002249052046009700F0ABFA002816
:109FB0000DD12068006840070BD501212B460022F7
:109FC00089052046009700F09DFA002801D0032063
:109FD000F8BD2020A067E067266660342675002063
:109FE000F8BD0000FFFFFF01F8B5184CC826E07867
:109FF000002829D16079002826D101206071144DF4
:10A00000686B002700281ED0686BC821081A15E06D
:10A010001048E168405C616988470F480A21008860
:10A0200048430E490880E068401CE060E068C828AA
:10A0300000DBE760696BC820401A761EE168814248
:10A0400001D0002EE4DC6771F8BD00005400002050
:10A0500000000240140D00203401002046010020C1
:10A0600070B5224CE07800283FD1207900283CD1FF
:10A07000012020711E4EF16900250906002933DAFE
:10A080002156625791420AD1F06940062CD5A07939
:10A09000002829D0A5712089401C208124E0A179C5
:10A0A000002903D1A0710A2000F091FD0020205664
:10A0B000CC2148430F494218206912181279B26224
:10A0C000401C00222061A256CC235A438958814269
:10A0D0000ADC25612078401C207020780E2800D1F1
:10A0E0002570A078401CA070257170BD5400002020
:10A0F00000380140EC01002010B5806A00220146C2
:10A1000040314A834A82FDF7DFFE10BD70B5846A94
:10A11000A06FE56F2168896800260906002906DA24
:10A12000212804D152200653204600F06BF8206805
:10A130008068400606D5222D04D15A2006532046B9
:10A1400000F047F82046803001681022114301607A
:10A150002046FDF7B9FE70BD10B501460968806A5A
:10A16000096889061CD400225A210A5201680A682B
:10A17000FF2301339A430A6001688A68520852003B
:10A180008A6001688A6840239A438A602021C167F7
:10A19000016E012904D101680A6810239A430A60FC
:10A1A000016E012902D0FEF771F810BD5821095A3D
:10A1B000FDF788FE10BD10B5806A016E012902D03E
:10A1C000FEF765F810BD5821095A4908FDF77AFED7
:10A1D00010BD01680A68FF2321339A430A600168B1
:10A1E0008A68520852008A60016E012904D1016810
:10A1F0000A6810239A430A602021C1670021016682
:10A200004166704701680A68C0239A430A602021AA
:10A210008167704770B5164CE278002A0CD122791C
:10A22000002A09D10122E2700025C82903DC02229C
:10A23000A256002A01DCE57070BD0123E356CC2252
:10A2400053430C4AD1500123E356CC2673439B1849
:10A250000A460146181DFAF791FF6078401C6070AD
:10A2600060780E2800D16570A078401EA070E2E7EB
:10A2700054000020EC010020F8B504460168806815
:10A280002369E66918436369002533431843724A1A
:10A290000B68724E334003430B6021684868032308
:10A2A0001B039843E368184348602168A069914202
:10A2B00001D0236A18438B680B263602B34303434D
:10A2C0008B606749236867488B420CD1C068800760
:10A2D000800F06D0012839D0022835D0032821D19B
:10A2E0001EE001271FE060498B420AD1C0680C21A3
:10A2F000084027D0042829D0082825D00C2811D1BF
:10A300000EE093420ED1C16803208002014019D0B3
:10A3100001208002091A19D0091A15D0814201D1F1
:10A32000082700E010274F495048403986009342E3
:10A3300032D1002F0CD0022F0DD0042F10D0082FB7
:10A340007FD126E00027EEE70227ECE70427EAE7C3
:10A35000FDF7DCF806E00968C90605D4304603E0DD
:10A36000FDF7F4F8002872D062685100511881425C
:10A3700067D81103814264D3010E060250080023FE
:10A3800030185941FAF7CAFE03210902411A384A26
:10A3900055E00120C003E7E70122E369D2039342BD
:10A3A0002BD13B0000F0E7F90906090C4D114D4D8A
:10A3B0004D274D00FDF7AAF809E0FDF7B7F806E0D4
:10A3C0000968C90605D4304603E0FDF7BFF8002848
:10A3D0003DD0616840004A088018FAF789FE80B2D3
:10A3E0000146244A103991422BD8511C01400007E4
:10A3F000400F084329E01046EBE73B0000F0BBF9B3
:10A400000906090C2112212121232100FDF77EF8E4
:10A410000AE0FDF78BF807E00968C90606D4304664
:10A4200004E00EE0FDF792F8002810D061684A08B9
:10A430001018FAF75DFE80B201460E4A10399142BB
:10A4400003D9012503E01046F0E72168C860002029
:10A450006066A0662846F8BD00480040F369FFEF3B
:10A4600000380140401002400044004000093D0017
:10A47000FFFC0F00EFFF0000F8B5044641654030D7
:10A4800000262746028380373E602220E06725466B
:10A49000206F603500281CD01749C162216F174812
:10A4A0000863216F16484863206F8663236F606DD1
:10A4B0009C4613462168024660462431FCF70EFA9A
:10A4C000002806D0102038602E752020A0670120BB
:10A4D000F8BD2E7520680168FF220132114301602A
:10A4E00020688168012211438160206881684022D0
:10A4F000114381600020F8BD59A10008B7A10008F0
:10A500000DA10008FFB581B005460F460446603531
:10A510000A9E39E0701C37D0FCF788FB0499401A7A
:10A52000B04222D8002E20D02068016849072BD5E0
:10A53000C069C043000527D401202168C002086219
:10A5400020680168FF22A132914301602068816880
:10A550004908490081602020A067E06780342060BE
:10A5600000202875032005B0F0BD20680168FF2297
:10A57000A1329143016020688168490849008160E7
:10A580002020A067E067EBE72068C1693846884370
:10A5900005D0002103988142BCD00020E3E70121CF
:10A5A000F8E7000010B50449102009680862024865
:10A5B000FDF78CFC10BD0000AC16002001490D20F9
:10A5C000887070475400002010B507480A22018A9D
:10A5D00051434184FEF71AFAFEF732FBC8220349C1
:10A5E0000348FDF723FE10BD24010020140D0020B8
:10A5F000AC160020F8B53E4C002321783D4A1D469C
:10A60000082910D0072947D0062950D0052952D053
:10A61000042953D0032954D0002956D0012958D0F9
:10A6200002295AD05BE0A17800264A1F04E0314F8E
:10A63000BF5DFB189BB2761C9642F8DB66792779E2
:10A640009A195118E3786278C9188918C9194018FD
:10A65000C0430006000E1AD1012E14D0022E16D1CE
:10A6600025482449C018FAF789FD01F08DFF6420C0
:10A6700000F0A6FABFF34F8F21492048C860BFF30E
:10A680004F8F00BFFDE759081046FFF7ABF9257063
:10A69000E570A570A571F8BDA1795054491CC8B2E8
:10A6A000A071A178491F8842F5D1082001E06070AF
:10A6B00007202070F8BDE0700620FAE760710520E1
:10A6C000F7E7A070E5700420F3E7552807D10120D3
:10A6D000EFE7AA2803D10220EBE7032803D0257077
:10A6E000E570A570F8BD032020702071F8BD000052
:10A6F0001C010020C0140020DC0D00200400FA051D
:10A7000000ED00E010B5024A024900F0E5F910BD85
:10A71000C1B800087C0100202021020C01D01021CA
:10A720001046020A01D010460839020901D010462D
:10A73000091F820801D01046891E420801D0881ED8
:10A740007047081A7047F8B5040C8BB2264682B2DF
:10A750005E430D0C1046370C584336048019002117
:10A76000794116466E43370C3604801979412646E6
:10A770006E438919F8BD30B47446641E2578641C94
:10A78000AB4200D21D46635D5B00E31830BC184746
:10A790004900CA020243100000D004204A0D01D033
:10A7A00001221043044A490D914201D1022108437C
:10A7B000012800D105207047FF0700008307FF2212
:10A7C000DB0E9A408907090E9940002808DB8308B0
:10A7D00009489B001B18186890430843186070478D
:10A7E0000007000F0838830804489B001B18D8692D
:10A7F00090430843D861704700E400E000ED00E0BA
:10A80000BFF34F8F04490348C860BFF34F8F00BFA9
:10A81000FDE700000400FA0500ED00E0F8B504468D
:10A820004F1EC8000838211815461E46086849689A
:10A830003A4606239A4310D02A463346FAF762FE78
:10A840003A46D200083AA3181A687F1E5B68FAF7E6
:10A85000A7FD06223B469343EED1022F23D0042FBF
:10A8600011D0062F2FD12A463346FAF74BFEE36A62
:10A87000A26AFAF795FD2A463346FAF743FE636A61
:10A88000226AFAF78DFD2A463346FAF73BFEE36962
:10A89000A269FAF785FD2A463346FAF733FE636963
:10A8A0002269FAF77DFD2A463346FAF72BFEE36864
:10A8B000A268FAF775FD2A463346FAF723FE636865
:10A8C0002268FAF76DFDF8BD002210B51346104658
:10A8D0000149FAF77FFE10BD0000F03F10B5FAF70E
:10A8E0005FFD10BD002210B5134610461146FAF761
:10A8F00071FE10BD10B50721024A00200907FAF7C2
:10A90000E1FE10BD01030000034A10B5002011074D
:10A91000FAF7D8FE10BD000001FDFFFF02E008C8F5
:10A92000121F08C1002AFAD170477047002001E0C9
:10A9300001C1121F002AFBD17047000001490860C5
:10A94000704700008001002008B5002168460170B2
:10A950006B46012202212C2000F052FF02216846A2
:10A9600001706B4601222C2000F04AFF08BD000058
:10A9700038B504466D20694608706B4601220749C8
:10A980002E2000F03DFF0649002C01D0054A00E0D2
:10A99000054A2E2000F01AFF38BD0000060800000E
:10A9A00006180000070600000716000038B5044628
:10A9B0006B4602220021362000F0EEFDB321230079
:10A9C000FFF7D9FE0E0F08153A3A3A3A1C273A3AE1
:10A9D0002F34483A00216846017040784108490008
:10A9E00014E06946087880088000401C04E069464D
:10A9F000087880088000801C08701DE06846027896
:10AA00000A40483202704178802001436846417014
:10AA100012E0684602780A40027040784106490E0A
:10AA2000F4E7694648780221084303E0694648781C
:10AA3000FD210840694648706B46012200213620FE
:10AA400000F0DEFE012200AB11463620013300F09B
:10AA5000D7FE38BD69460878CF21084069462030C6
:10AA6000CAE708B5032168464170012101706B46B1
:10AA700002220021362000F0C3FE0122D20306216B
:10AA80002D2000F0A3FE012000F09AF80120FFF72E
:10AA90008DFF08BD08B5020A69464A7008706B460A
:10AAA000022204212D2000F0ABFE0320694608702D
:10AAB0006B46012206212D2000F0A2FE00206946EF
:10AAC00008706B46012206212D2000F099FE0A2114
:10AAD0002D2000F047FD08BDF8B516460F46044688
:10AAE000002503E03946B047641C6D1C207800281F
:10AAF000F8D12846F8BD0000F8B54A002B4B520D9E
:10AB0000D6182B4A0C460546142E2BDA002E12DAE4
:10AB1000284BFAF745FC00221346FAF7B5FE40D25F
:10AB2000002C03DA0124E40700253AE020462843FC
:10AB300037D0214C14E0214F0B46F7403B402B43CC
:10AB400031D01C4BFAF72CFC00221346FAF79CFE7E
:10AB500027D2002C03DD01200005F0400419BC437E
:10AB600000251EE0332E1EDC33460027143BFF4336
:10AB7000DF40384217D00F4BFAF7BCFC00221346D7
:10AB8000FAF782FE0DD2002C0ADD142E0CD03420F0
:10AB9000811B012088404019A84200D2641C054650
:10ABA000BD4321462846F8BD641CF9E701FCFFFFC0
:10ABB0009C7500883CE4377E0000F03FFFFF0F00EB
:10ABC0007D2110B5C900484300F001F810BD0021F7
:10ABD00040E000BF00BF00BF00BF00BF00BF00BF1C
:10ABE00000BF00BF00BF00BF00BF00BF00BF00BF6D
:10ABF00000BF00BF00BF00BF00BF00BF00BF00BF5D
:10AC000000BF00BF00BF00BF00BF00BF00BF00BF4C
:10AC100000BF00BF00BF00BF00BF00BF00BF00BF3C
:10AC200000BF00BF00BF00BF00BF00BF00BF00BF2C
:10AC300000BF00BF00BF00BF00BF00BF00BF00BF1C
:10AC400000BF00BF00BF00BF00BF00BF00BF00BF0C
:10AC500000BF491C8142BCD37047FFB581B01E467E
:10AC60000F46040026D00B9903980143A06A39438C
:10AC7000826807209047002818DB0A99A06A3143B0
:10AC8000826806209047002810DB25462035A979E8
:10AC9000032F01D908200143032E01D904200143C9
:10ACA000A06A826809209047002806DA0120C04384
:10ACB00005B0F0BD0020C043FAE7384600F000F9C7
:10ACC0002060304600F0FCF860600A9868700398D5
:10ACD000A870EF702E710B9868710020E8E70000F3
:10ACE000F7B50446002090B000900190002C05D0EC
:10ACF0006A46062101F082FC062803DA0020C043E0
:10AD000013B0F0BD68464078010268460078000440
:10AD10000918684680780818FAF710FD0546684655
:10AD20000391007901026846C0780004091868465A
:10AD300040790818FAF702FD032206460F469207EB
:10AD40005C4BFAF7A1FD07D200225B4B3046394637
:10AD5000FAF7CAFB06460F4603229207554B2846D0
:10AD60000399FAF791FD07D20022534B2846039925
:10AD7000FAF7BAFB054603912068FAF7DFFC0246B2
:10AD80000B4630463946FAF725FC07460A2007915C
:10AD9000205EFAF7BFFC3A46079BFAF7B3FB06467C
:10ADA00008200991205EFAF7A3FC0021C943FAF7B5
:10ADB000EAFAFAF741FD3246099BFAF7F1FA0691F1
:10ADC00008906068FAF7BAFC02460B4628460399D9
:10ADD000FAF700FC05461A200E46205EFAF79AFCA8
:10ADE0002A463346FAF78EFB0C9009911620205E16
:10ADF000FAF790FC099B0C9AFAF7D2FA05910A909F
:10AE00002A46334638460799FAF77CFB059B0A9A8F
:10AE1000FAF778FB05910A901420205EFAF77AFC85
:10AE20003A46079BFAF76EFB07461C200791205E07
:10AE3000FAF770FC2A463346FAF764FB0E900B9142
:10AE40001820205EFAF766FC0B9B0E9AFAF7A8FA18
:10AE50002A463346FAF756FB0B910E902069FAF713
:10AE600059FC0B9B0E9AFAF79BFA2A463346FAF7DF
:10AE700049FB05460E46E068FAF74CFC2A46334685
:10AE8000FAF78EFA3A46079BFAF78AFA059B0A9A6E
:10AE9000FAF786FA01229207084BFAF733FB0246CB
:10AEA0000B46129C0898069903C411980CC0002008
:10AEB00026E70000FFFF5F4100007041E17A843F18
:10AEC00000B50121C9040300FFF755FC081A050865
:10AED0000B0E1114171A0320C00400BD0720C00474
:10AEE00000BD0F20C00400BD1F20400300BD3F2057
:10AEF000400300BD7F20400300BDFF20400300BD94
:10AF0000084600BDFEB5264F0D4604000FD0002DAB
:10AF10000DD0264600202036B071F07129680D2032
:10AF20008847002801DA7800FEBD102801D0384695
:10AF3000FEBDA562E968002901D028208847204687
:10AF400000F030F80028F3DBA06AA52182680E200B
:10AF50009047A06A962182680F209047A06A02213C
:10AF6000826862209047A06A002182680E20904784
:10AF7000A06A002182680F209047717930200191EA
:10AF800000900623202201212046FFF766FE0028BC
:10AF9000CEDB204600F0AEF80028C9DB0020FEBD65
:10AFA000FFFFFFFF10B586B0044614216846FAF78C
:10AFB000FEF8002C7ED0A06A122143686A46102059
:10AFC0009847122877D16846007801220101684627
:10AFD000407812030009081843492081884201DDA6
:10AFE000801A20816846837840780007000D181881
:10AFF0006081884201DD801A608168460079012203
:10B0000001016846C07812050003091868464079B6
:10B01000000908183549E060884201DD801AE060C7
:10B02000684640790007030B6846807900021B18C8
:10B030006846C07918182061884201DD801A2061B5
:10B040006846417A007A0002081802B228480121B5
:10B050000904A282824201DD521AA2826A46D37A90
:10B06000927A12029A1812B2E282824201DD521AD8
:10B07000E2826A46537B127B12029A1812B2228332
:10B08000824201DD521A22836A46D37B927B1202EE
:10B090009A1812B26283824201DD521A62836A46B2
:10B0A000537C127C12029A1812B2A283824204DDEF
:10B0B000501A01E00BE008E0A083A06A0168282094
:10B0C0008847002806DA0120C04306B010BD0020E2
:10B0D000C043FAE7C011C0072034002800D0802008
:10B0E00060710020F1E70000FF070000FFFF07008C
:10B0F000FF7F000010B5040009D0A06A0721826814
:10B1000008209047002805DA0120C04310BD002028
:10B11000C04310BD072020342070002010BD000067
:10B12000FEB504460020019000906079734940000C
:10B130000E5A61782578491E7148CFB20163042DFB
:10B1400077D0072D75D000210291217801736C49C9
:10B15000E379012292058969002B6CD091438161CA
:10B160006748217A4173217A82698907890B0A43EA
:10B1700082610021042000F034FB324661492E2018
:10B1800000F024FB3846FFF7F3FB5F4E0522705DAD
:10B19000810040185D49431807212B2000F030FB47
:10B1A0005B49029801220B180B21282000F028FB94
:10B1B000705D584980000A580C21282000F011FBCE
:10B1C000E079554980004018A1794900425A02218E
:10B1D000272000F0FBFA51487E00825B04212720E3
:10B1E00000F0F4FAE079002829D0A07804282CD0C7
:10B1F00028206946087220220621272000F0E6FA5E
:10B2000002AB01222621272000F0FAFA4449380136
:10B210004018E178890042580821272000F0E1FA1F
:10B22000A17A601C627A0902114313D016E000E093
:10B2300001E0012188E71143F608816190E764226B
:10B240000621272000F0C2FAE0E7102069460872C4
:10B250000246D1E733490172090A4172417A007A04
:10B260000A0202432021272000F0B0FA2E4F0C21C1
:10B2700023203A6800F0B5FAF019828804212320CF
:10B2800000F0A4FAA07900280BD0E0792749012228
:10B2900043180021212000F0B3FA0320019001207F
:10B2A00000902A07120F10010243607800218007E6
:10B2B000000B02430198000502430098400402433A
:10B2C0002079C006400902436079C00602431F206E
:10B2D00000F087FAA0786178012308430204084847
:10B2E000DB030261E179490319430A43026100214A
:10B2F000082000F076FA0020FEBD000030C70008EC
:10B30000B001002004280000D8C600082400002056
:10B3100042000020E0C6000800C700080CC7000873
:10B3200010C7000841100000F8C6000844000020C3
:10B3300038B50C4607498A8B002102432C2000F0C7
:10B3400045FA684604706B46012206212C2000F065
:10B3500057FA38BDB001002010B5FFF7F5FA10BD5F
:10B3600010B504460421362000F0FCF80121C90282
:10B37000002C01D0084300E0884302460421362017
:10B3800000F02FFA10BD000038B540206946087063
:10B3900000210E2000F0E6F80446002211460E209F
:10B3A00000F01FFA6B46012200210D2000F028FA60
:10B3B000074A00210F2000F014FA00F0EDF92246B0
:10B3C00000210E2000F00DFA02480021017338BD63
:10B3D000F8FF2724D0010020FEB505460420694669
:10B3E0000870514C0020607521462031206348715F
:10B3F0000873A0836063A06300F0C8F84B4E206020
:10B4000002E000F0C3F82060B042FAD10020FFF75C
:10B41000CDFA00F0BBF8464E20603078242801D9E0
:10B42000243806E00621F9F763FE0622101A4001CF
:10B430000843020601040A4301020A430243B260C0
:10B44000706000211E2000F0CCF900F09FF8206011
:10B450006B4601220021242000F0D2F91E20FFF7C4
:10B4600019FB86B2300AA0730420FFF713FB0746CE
:10B4700000F08CF820603806000E0DD002206946DE
:10B48000087101AB012212212D2000F0B9F9A08B27
:10B49000012109030843A08300F078F8206006200A
:10B4A000FFF7F8FA60600720FFF7F4FAA060F006F3
:10B4B000C00E207501D110202075C0B200F0DCF95B
:10B4C000E80707D0FFF7CDFAA08B0121C902084396
:10B4D000A0830AE00521362000F02EF81549084027
:10B4E00002460521362000F071F90120FFF75EFACF
:10B4F0000021042000F036F8A0610021262000F091
:10B5000031F815218903084302460021262000F066
:10B5100068F900222621362000F058F900F036F8AC
:10B5200020600020FEBD0000B00100203001CADE16
:10B5300018000020FFFD000038B5094C89B280B228
:10B540006B46022200F028F8002806D168464078B1
:10B55000010268460078081884B2204638BD000011
:10B56000FFFF000038B50024E44389B280B26B4687
:10B57000042200F011F8002806D103216846435C3C
:10B580002202D418491EFAD5204638BD10B5002134
:10B590000846FFF7E7FF10BD38B5002909D0402461
:10B5A00020436C462070C8B27F2906D86070022004
:10B5B0000AE069460870012006E0802420436C46BA
:10B5C0006070C809A0700320694600F0B7FF38BD5D
:10B5D00010B5144603460A4621461120FFF7DCFF4A
:10B5E00010BD10B50346052200211520FFF7D4FF3A
:10B5F00010BD10B50346052200211720FFF7CCFF30
:10B6000010BD38B5054600206946087000F0C4F842
:10B61000FF2401342246002D01D003221202002112
:10B620000D2000F0D3F8002D13D06B46012203212A
:10B630000F20FFF7B1FF68460078000709D5FFF734
:10B64000A3FE224600210D2000F0C0F80020C043D8
:10B6500038BD002038BD10B5024601210A2000F097
:10B66000C0F810BD10B5044600211A20FFF77AFF7C
:10B67000000D22030005120B024300211A2000F0E6
:10B68000B0F810BD10B5024602492E2000F09EF819
:10B6900010BD000004180000F8B505466B460122F5
:10B6A00003210420FFF778FF0126114C3607002DF7
:10B6B0000DD02A4600210C2000F088F86946087851
:10B6C0001021084369460870A069304307E06946C5
:10B6D0000878EF21084069460870A069B0430B461E
:10B6E000A06101220321042000F08AF8F8BD0000C7
:10B6F000B001002010B502460021182000F066F8C5
:10B7000010BD0000F8B50746002568460570B8076B
:10B71000204C2E4600280ADA8020694608706B46C5
:10B72000012200210D2000F06BF801202073F807A2
:10B730006946087821D006210843694608706B469F
:10B74000012200210D2000F05BF803210F20FFF7FC
:10B75000F3FE8121C900084219D0402069460870D3
:10B760006B46012200210D2000F04AF80020FFF76F
:10B77000F7FD00252673ED4309E0022108436946E1
:10B7800008706B46012200210D2000F039F8284690
:10B79000F8BD0000D00100201CB56B46012203213A
:10B7A0000F20FFF7F9FE684600784022C1091040DB
:10B7B000C9014000814208D0012069460871024653
:10B7C00001AB03210D2000F01BF81CBD08B56B4632
:10B7D0001A70120A5A7089B280B2022200F010F870
:10B7E00008BD38B500236C46E254120A5B1C042BDA
:10B7F000FADB89B280B22346042200F001F838BD9A
:10B8000038B58024002909D0C02528436D4628700A
:10B81000C8B27F2907D86870022009E02043694632
:10B820000870012004E020436870C809A870032054
:10B83000694600F02DFF38BD10B5144601231218DB
:10B840009B029A4202D90020C04310BD0B46821EC3
:10B8500021460920FFF7D4FF002010BD10B5054A8E
:10B860008905126901430A4300210820FFF7B9FF47
:10B87000002010BDB001002038B504466B460122FF
:10B880000E212B20FFF788FE68460078E10640096C
:10B890004001C90E0143684601706B4601220E212A
:10B8A0002B20FFF7ADFF38BD10B5002142541C0618
:10B8B000120A22431B0A491C0429F7DB10BD0000B1
:10B8C00013B501231A4669460248FCF7E1FC0098CB
:10B8D0001CBD0000AC1600207CB50024254668463F
:10B8E000FFF77FFE04206946220E2D021543220237
:10B8F0000C5C1443401EF7D5204629467CBD7CB520
:10B90000002425466846FFF774FE04206946220E8F
:10B910002D02154322020C5C1443401EF7D520462D
:10B9200029467CBDFBF790F9FEF7EAF8FDF782F8AF
:10B9300041494248002522C005608561C5614049F2
:10B940000562C1600838FBF71BFBFDF75FF8FDF7E8
:10B9500077F9FDF713F9FDF725F8052601223607DB
:10B96000D1033046FBF75BF9FDF73AFEFCF70EFF1B
:10B97000FAF7F0F9FAF7BEF9FCF70CFD0721B0155C
:10B98000FFF7D6FCFFF7E8FC2E4C0A21208A0122A3
:10B990004843608411033046FBF741F92748C82229
:10B9A0002949C830FCF742FC284F294E207900284D
:10B9B0003FD0607800283CD0FEF7A2F82571FAF756
:10B9C000F5FB20700F280AD9012211033046FBF73E
:10B9D00026F9FEF7E3F900220121090309E001221B
:10B9E00051033046FBF71BF9FEF7D8F9002201217D
:10B9F00049033046FBF713F9FCF7F4FD608C00288F
:10BA000001D0401E60841348618C00780843CDD17A
:10BA10003878002801D00328C8D10121C902304656
:10BA2000FBF7F0F80028C1D101210846FBF7BCFB69
:10BA3000BCE7FCF7D7FDB9E7007C0040E415002027
:10BA4000FFFF000024010020140D002081000020D1
:10BA5000000400505A00002010B586B01748FBF7CC
:10BA600012FA14216846F9F7A2FB1548009003204A
:10BA7000019000200290052069460007FBF706F8B8
:10BA800069461048FBF702F869460F48FAF7FEFFCF
:10BA900001210846FBF788FBFF2401342046FBF711
:10BAA0005BFB0A4908680422104308602046FBF744
:10BAB00063FBFBF769FB06B010BD0000E415002036
:10BAC000FFFF00000004005000080050007000401C
:10BAD00010B50122920217491748FAF7C7F915481D
:10BAE000164902888A4224D00180FF2101318180D9
:10BAF000FF21F531C1800A21018100211E224181EF
:10BB0000D24382810122C28181831E23C386022304
:10BB10000387782343878287C28702464032118495
:10BB200051849184C183918014238382118200F017
:10BB30002BFD10BDDC0D002000FC0008AA55000004
:10BB4000F0B51FB496B084460C460246199D18986D
:10BB50000390490068006300490840080193002AE7
:10BB600001D0012600E000269E19FE4BF6185B105E
:10BB70009E422BD36E00039F0296002F00D0012718
:10BB8000F719F84EF84BBE199E421FD3039E034689
:10BB9000F64F334309D03B469C4201D1002A04D0E2
:10BBA000019B002A05D0012604E0002039461BB085
:10BBB000F0BD00269E19EE4B9E4207D8039F029EC1
:10BBC000002F00D00127F6199E4207D92B46604668
:10BBD0002146189AFEF782FE1BB0F0BD0023002C10
:10BBE00029DAE44EB04226DAE34EB04201DB02230A
:10BBF00021E0DE4EB0421EDBE04E070DBE19142ED2
:10BC000009DD3427BF1B039EFE400196BE40039F03
:10BC1000BE420BD00FE0039F002F0CD11427BF1B97
:10BC20000646FE400196BE40864204D1019BDE07D7
:10BC3000F60F02239B1B0E46164318D1002D16DA71
:10BC4000002C03D0022B01D0012B06D00220FEF7DE
:10BC500075FEFEF739FE1BB0F0BD0220FEF76EFE4A
:10BC6000FEF732FE0122D20751401BB0F0BD039E09
:10BC7000002E61D1BF4EB04220D1C148844201D1D3
:10BC8000002A08D0B948814209DB002D10DB189842
:10BC900029461BB0F0BD0020B4491BB0F0BD002DFB
:10BCA00006DA01222946D207189851401BB0F0BD90
:10BCB000B4497944086849681BB0F0BDAB4FB8423D
:10BCC00025D1002D1FDA002904D0B14212D1002A5B
:10BCD00009D018E0002A72D1A649E20F0020D2074D
:10BCE00011431BB0F0BD0020E20F0146D207114303
:10BCF0001BB0F0BDB14206DA234600203946F9F701
:10BD000069FC1BB0F0BD104621461BB0F0BDB1422E
:10BD100012DA0126B607B54203D12346104619466A
:10BD2000FEE3994EB54207D1261E05DB104631468B
:10BD300000F040FC1BB0F0BD67007F081646002AEB
:10BD400040D100290AD08B4A914229D1002C0EDD26
:10BD5000002D1CDB002011461BB0F0BD022B16D0BD
:10BD6000002C14D0012B12D1002C14DB0FE0002C7E
:10BD700028DA002D09DB012B03D000207D491BB000
:10BD8000F0BD002081491BB0F0BD012B03D0002085
:10BD900001461BB0F0BD00200121C9071BB0F0BD5A
:10BDA000724A91420ED1002C01DA002B17D0022BDF
:10BDB00006D00020C043F9F7ADFC1BB0F0BD90E207
:10BDC0000120F8E7E217521C94461A4307D00022DC
:10BDD0000892664C62465B1E1A4307D009E00120B8
:10BDE000FEF7ACFDFEF77EFD1BB0F0BD0022644CFB
:10BDF0000892674A90427DDD664B674A98421FDD94
:10BE0000914202DC002D05DB4DE05848814217DBF2
:10BE1000002D48DD0220FEF791FDFEF76BFD054683
:10BE20000E460022534B21460898F9F76BFB084653
:10BE300071004908C00FC007014328461BB0F0BD80
:10BE4000914215DA002D2EDA0220FEF777FDFEF77B
:10BE500051FD05460E460022464B21460898F9F74B
:10BE600051FB72005208C80FC0070243114617E089
:10BE70003E4B994223DD002D15DD0220FEF75EFDCD
:10BE8000FEF738FD05460E4600223A4B214608983B
:10BE9000F9F738FB084671004908C00FC007014395
:10BEA00028461BB0F0BD0220FEF748FDFEF72CFD32
:10BEB00049004908E20FD20711431BB0F0BD002230
:10BEC00030463946F9F710FB012205460E46D243AB
:10BED000F9F7F8FB314A324BF9F70CFB2A463346A7
:10BEE000F9F710FB0022284BF9F704FB07462A4616
:10BEF000334600E064E0039110461946F9F702FB6F
:10BF00003A46039BF9F7FEFA0746032209915207C6
:10BF1000244B28463146F9F7F5FA07910C90224A4E
:10BF2000204B38460999F9F7EDFA074601911F4A67
:10BF30001F4B28463146F9F7E5FA3A46019BF9F7D7
:10BF4000D3FA07460B460246099107990C98F9F770
:10BF500027FA00250E462846079B0C9AF9F7C4FAE3
:10BF60003A4627E0FFFF1F00FFFF0F000000F03FF1
:10BF70000000E0FF0000F07F0000404301FCFFFFF5
:10BF80000000F0BF5A0B00000000E03F0000F0FF8F
:10BF90000000E0410000F043FFFFEF3F55555555CD
:10BFA0005555D53F4715F73FFE822B6544DF5DF8B9
:10BFB0000BAE543E099BF9F79DFA02460B4652E13F
:10BFC000012500202D05A94207DA352230463946E1
:10BFD000F9F778FB06463420C0430A151218FE48CC
:10BFE000101803900803FD49000B01430F46FC495C
:10BFF000884201DC002003E0FA49884202DA01208D
:10C00000119005E0002011900398401C7F1B0390C5
:10C0100011980597C200F4480F927844801843683D
:10C020000268394630460D930292F9F75DFA07919E
:10C030000C9030460D9B029A0599F9F7B1F902462A
:10C040000B460020E549F9F7C5FA09910490079BD2
:10C050000C9AF9F757FA129000201090E3480D4619
:10C06000784400680E90012178104907084311991F
:10C070000D9B890440180121C90447183946029ACA
:10C080000E98F9F731FA3246059BF9F733FA024672
:10C090000B4629461098F9F735FA064602913B46B9
:10C0A00029460E9A1098F9F72DFA079B0C9AF9F782
:10C0B00021FA3246029BF9F717FA099B049AF9F71D
:10C0C00021FA0591129A0A902B4610461946F9F763
:10C0D00019FA06460246C6480F460B460621784422
:10C0E000FEF79CFB32463B460091049010461946F1
:10C0F000F9F708FA009B049AF9F704FA06460F4686
:10C100002B461946129A1098F9F74AF9059B0A9A94
:10C11000F9F7F8F932463B46F9F742F9109A0791D8
:10C1200004902B4610461946F9F7ECF9B14E00225F
:10C13000334609910290F9F733F9079B049AF9F70E
:10C140002FF900200746024633460091F9F7CCF953
:10C15000099B029AF9F7C8F9079B049AF9F7CAF9FB
:10C1600006460D913A462946009B1098F9F7CAF900
:10C1700007910C902B463046129A0D99F9F7C2F9A7
:10C1800005460E463A46009B05990A98F9F7BAF912
:10C1900033462A46F9F704F902460B460746099149
:10C1A00007990C98F9F7FCF800250E462846079BDE
:10C1B0000C9AF9F799F93A46099BF9F79BF9074662
:10C1C0000722099152078C4B31462846F9F79AF914
:10C1D00007910090894A884B38460999F9F792F9F6
:10C1E00007460191864A874B31462846F9F78AF976
:10C1F0003A46019BF9F7D4F8834B7B440F9A9B187E
:10C200001A685B68F9F7CCF8029009910398F9F77E
:10C2100081FA05910490099B029A07990098F9F711
:10C22000BFF87A4B7B440F9A9B181A685B681746D5
:10C230000393F9F7B5F8059B049AF9F7B1F80E46A0
:10C240002846059B049AF9F74FF93A46039BF9F7FC
:10C250004BF9079B009AF9F747F9099B029AF9F7FE
:10C2600049F902460B46199900200C900F46189880
:10C27000F9F748F9029104903B460C9A19991898DD
:10C28000F9F732F92A463346F9F73CF9029B049A4A
:10C29000F9F786F809910E902A46334639460C98EC
:10C2A000F9F730F906460F46099B0E9AF9F778F828
:10C2B000574A0D46914220DB5242AA18024310D140
:10C2C00032463B46F9F710F904900391514A524B1C
:10C2D00009990E98F9F764F8039B049AF9F7D4FAD0
:10C2E0001ED20220FEF72AFBFEF704FB4900490894
:10C2F000E20FD20711431BB0F0BD6A00474B520852
:10C300009A420DD3464AAA18024300D0CBE53246E2
:10C310003B46F9F7E9F8099B0E9AF9F7B5FAF5D912
:10C320006800002340082C490393020D3D4B52182E
:10C33000984223DD01200005521CD04042195000D4
:10C34000400D401838497944096813468C463749EE
:10C35000C1408B4312030121120B0905511814220D
:10C36000101AC1400391002D01DA48420390624641
:10C3700030463946F9F7B8F806460F4632463B468E
:10C3800009990E98F9F70CF800252A46284B2846FB
:10C390000591F9F7B7F807910C90264A264B2846E5
:10C3A0000599F9F7AFF80091029032463B462846CE
:10C3B0000599F9F799F8099B0E9AF9F79BF81F4A26
:10C3C0001F4BF9F79FF8009B029AF8F7E9FF074621
:10C3D0000B460246099135E001FCFFFF0000F03FEB
:10C3E0008E9803007AB60B006A070000AC070000C5
:10C3F000D60600000000084009C7EE3FFD033ADC06
:10C40000F5015B14E02F3EBEAA0500007005000098
:10C4100000009040FE822B654715973C00CC904071
:10C4200000346F3F0000E03FC6040000FFFF0F0034
:10C43000432EE63F396CA80C615C20BEEF39FAFE52
:10C44000422EE63F07990C98F8F7AAFF05460E46DC
:10C45000079B0C9AF9F748F83A46099BF9F74AF80E
:10C4600009912A4633460E9010461946F9F74AF8C4
:10C47000074602462F480B46059105217844FEF7F2
:10C48000CDF93A46059BF9F73DF82A463346F9F7C8
:10C4900031F80746019128463146099B0E9AF9F773
:10C4A00031F8099B0E9AF8F77BFF012304910C9059
:10C4B00000229B0738460199F9F716F805910E906E
:10C4C0003A4628463146019BF9F71CF8059B0E9A1F
:10C4D000F9F780F8049B0C9AF9F706F82A463346D8
:10C4E000F9F702F80022144BF9F704F8064603980E
:10C4F0000D46000541190915002912DC3046294670
:10C50000039AF9F7DFF8FEF743F9042801D1FEF7A3
:10C51000FBF930462946039AF9F7D4F8064601E0BC
:10C5200004E029180B46324621460898F8F7EAFF3E
:10C530001BB0F0BD680300000000F03FF0B58C4672
:10C5400000251026052109078E620E4C08E067467B
:10C550007F5DE760A768FF07FCD0E7681F706D1C70
:10C560008542F4DB0020074606E0E760A568ED079A
:10C57000FCD0E5681D54401C9042F6D38E6100202B
:10C58000F0BD00000030014070B572B60124074DC7
:10C59000A40221462846F9F74FFC002804D0224681
:10C5A00003492846F9F7ECFC62B670BD00FC0008B0
:10C5B000DC0D0020F8B506460C46F9F773FA051EA7
:10C5C0000F4600D00120014349000B484908411A99
:10C5D000C90F0DD0002E01D0012100E000210C4335
:10C5E00061004908401AC00F02D10120FEF7A6F9E8
:10C5F00028463946F8BD00000000F07FF8B5154622
:10C600000E460746002407E03819C0B200F008F8CB
:10C61000641C2870E4B26D1CB442F5D33046F8BDFA
:10C6200010B50446FBF77AFFEE20FBF74AFFFBF755
:10C63000AEFF2046FBF745FFFBF7A9FFFBF76EFFB8
:10C64000EF20FBF73EFFFBF7A2FF0020FBF70CFFFC
:10C650000446FBF77EFF204610BD704770B50D46BF
:10C660000446FBF75BFFEE20FBF72BFFFBF78FFF8A
:10C670002046FBF726FFFBF78AFF2846FBF721FF42
:10C68000FBF785FFFBF765FF0A20FEF7A0FA70BDF8
:10C69000F0B50025102605279C463F070B46BE62D5
:10C6A0000C4C06E0595DE160A168C907FCD0E16867
:10C6B0006D1C8542F6DB002007E06146095CE16005
:10C6C000A168C907FCD0E168401C9042F5D3BE6167
:10C6D0000020F0BD0030014000000102030400050D
:10C6E000405C0000A05C0400C06C0800805C04009A
:10C6F000E03F1E00E07D1E0007A9022570889B8890
:10C700000A001600010006000100020087008D00EB
:10C710002D001A3152001A339A001A351D011A37AA
:10C720006B003B31BE003B335E013B3596023B372D
:10C73000000099599959EB518F421E45142E0080E3
:10C74000EB51F5283333E13A703DE13AC235852BA0
:10C75000C2353333C235C235AE47E13A5138A33022
:10C760005138000000000000000001020304060729
:10C770000809030406080C1018203000000000010E
:10C780000203040000000000000000000000F03F71
:10C79000000000000000F83F000000000000000062
:10C7A0000000004003B8E23F00000000000000006D
:10C7B00006D0CF43EBFD4C3E033333333333E33FFB
:10C7C000FFAB6FDBB66DDB3F4D268F515555D53F27
:10C7D00001411DA96074D13F65DBC9934A86CD3FF5
:10C7E000EF4E454A287ECA3F3E5555555555C53FE3
:10C7F00093BDBE166CC166BF2CDE25AF6A56113FD5
:10C80000F16BD2C541BDBBBED0A4BE726937663ED6
:10C81000000000000000000038C8000800000020F0
:10C82000840100006C5B000898C8000884010020A7
:10C83000541A00002CA900080124130704380D091C
:10C840001E080540082609104008560A131D043B1F
:10C8500008BE0516D8BC40100852010336C8420372
:10C86000605C121B0202C5140901022281F01F66DE
:10C8700081049889968696798215980398149887EA
:10C880009674977882439788967197778249D901F1
:08C8900045294B92049220009F
:04000005080050C1DE
:00000001FF
